:020000041100E9
:10300000002373B52B4D2C4C28006361022601F080
:1030100065FA4021FE2221742800284B009601F019
:10302000AFFA002836D1217CFF222800244B0096DD
:1030300001F0A6FA00282DD1224BA2899A4226D16E
:10304000E389214A93420DD1204B6361204B2268D2
:10305000002A03D1002B01D043CB43C4280001F048
:103060007BFA73BD1B4A934201D00023EFE71A4B52
:103070001A4A1B68934206D9C02304222800217CE7
:103080009B0001F0F3FA114B6361154BDFE700235E
:103090002374EAE7CC233821AC2228009B01217459
:1030A00001F0E4FA0028F2D10E4B63610E4BE3818C
:1030B0000E4BCCE7BC44FF1F6C64FF1F7864FF1FFE
:1030C0007A64FF1F5959000083050000094300116D
:1030D00048BF0011821500009064FF1F8713000095
:1030E00054BF0011C1430011AAAAFFFF3CBF001149
:1030F000F7B5164B0192C318021D002000938823D8
:103100005B05D3181B685C1C1AD09CB2402C18D8E5
:103110008D781E0CAC466746CD782D023D43AE42FD
:1031200006D1019800280ED110000C70240A4C70B2
:1031300003249BB20733A343D218009B9A42DED3E9
:10314000FEBD4432F9E71000FAE7C046FC0F00006C
:10315000802213B503000324019189B25201073183
:103160009B18A14304305A1A88235B05C3181B68B7
:10317000591C03D190429241104016BD99B240298A
:1031800007D80B000733A343C0189042ECD30020AC
:10319000F3E74430F9E7134B134A1B68126810B584
:1031A000FA24934201D81A00F824104BE4021B6859
:1031B0009A4210D813000E4A12689A420ED3013375
:1031C00007D1F823DB029C4203D10A49054808F0E5
:1031D000ABFC200010BDFC24E402ECE7FE24E4027A
:1031E000F7E7C04600C0071100D0071100E0071143
:1031F00000F00711FFFFFF7FF0B59BB015000490B2
:103200000391402A00D9A0E006AB59801A80FFF74D
:10321000C2FF0400042816D9002206A9FFF768FFA0
:10322000052810D906AB1B88AB420CD1002D07D066
:10323000514B2A000499C01808F0CEFB002802D197
:1032400001201BB0F0BD06AB1D8020000699FFF7E2
:103250007FFF041E7BD1069B0793FFF79CFF802313
:103260005B01C618802307001B039E4201D3F8268A
:10327000F60288235B05F31801931B68013302D023
:10328000019808F059FB3D49019808F04DFC3B1DA1
:103290000293331D05938822029B52059B181B68DD
:1032A00008935A1C3CD044219AB20091402A04D879
:1032B0000320D11D814389B2009103991B0C8B42DD
:1032C00024D0402A22D80122300008A9FFF710FF9D
:1032D000021E1BD1380008A9FFF70AFF04000428CA
:1032E00031D9009A059B9B1880225201B218934253
:1032F00040D288235B05C118009A09A808F01CFC7D
:103300001D4B009A09A9F01808F036FC009A029BA0
:103310009446634402931A4B029AFB189A42BAD31A
:1033200088235B05FC1821680198013908F0FCFB33
:10333000200008F001FB039A07AB5A803000079980
:10334000FFF706FF0400002C03D1002079E70428D2
:10335000FBD988235B05E018069908F0E5FB0323F9
:10336000EA1C9A4300D16BE7034B0499E01808F07C
:1033700003FC65E70424ECE704000011FFFFFF7F76
:10338000F80F0000F7B505001400402A21D80027E7
:1033900001AE71803780FFF7FEFE042816D93A008F
:1033A0003100FFF7A5FE042810D93688BC420BD0A7
:1033B000BD4209D0221CB44200D9321C064B92B245
:1033C000C118280008F0B8FB30B2FEBDC04300B2FF
:1033D000FBE703204042F8E70400001137B5042260
:1033E00004000D0001A81649FFF7CCFF02000428D5
:1033F0000BD1019BA34208D3AB4204D0104901A8D2
:103400000195FFF7F9FE01203EBD0E4C2368200018
:10341000019308F091FA019920000139019108F017
:1034200083FB80235B01E418074B9C42EED104220E
:10343000034901A80195FFF7DFFE0020E4E7C0463D
:103440005555000000C007110000081130B589B0C3
:1034500008F032FA10226946254808F0F5F9254BA4
:10346000009A9A420ED1019B029A0F2B33D8002169
:1034700001240698013B08D2002900D00292029B49
:10348000013331D10023029325E0551CF2D1020013
:103490002100EFE710341022200004A908F0D4F92D
:1034A000029B013301D1069B0293882304995B059B
:1034B000C918059B06981A03120B049105928142C4
:1034C00003D02B4201D108F037FB019B013B019354
:1034D000019B002BDED1029B002B03D004930498A8
:1034E0004168084709B030BDE025014C2D03EFE7E6
:1034F0000000011150485936F7B50F4F0F4BFA6DC8
:1035000004001A4084235B001343FB65030010335F
:10351000019300252E00112008F0C6FB0322BB6E8C
:103520001340AB4002351E43202DF4D1019B40C413
:10353000A342EED1F7BDC04600F0004000FEFEFF02
:10354000802270B5AD4CAE4BD200002120001C6033
:1035500008F07AFC2300AB4A88331A60AA4B1A7829
:103560006E23002A00D01133E3620A232365A74BA0
:103570001878A74BA0630138E361C3B2032B01D8CD
:1035800010232362A34B37226361C823DB00A361AE
:1035900023008C331A60082336210F3AE518E163C3
:1035A00023646264E9670439251DE96725003B2629
:1035B000BC352E602500C0352B602500C4352A603F
:1035C00025000636CC352E602500083EC8352E6015
:1035D0002500D03529602100D4310B602100D8317D
:1035E0000A6021000225E0310D6025004221DC3512
:1035F000296025001B3EE4352E602500E8352B6050
:103600002500EC352A6022000525F43215602200E1
:10361000F032116022001831903211602200943291
:10362000136023003C2298331A60AF23DB00236031
:10363000794B2363032805D808F00EFC3302353795
:103640001523636096232100FA225B00A360E360E8
:10365000C8332361714BFC319200A3640A6062623B
:103660006F4A704DA2627322E2656D3A6265A2658F
:103670000232E5644A600221616696218900A166F2
:10368000626709210022E166A2676749674A684EBE
:103690002167E2673560032811D808F0DDFB960842
:1036A0009EA61023CDE70E23CBE70C23C9E720000D
:1036B0001A259C30056020000735A03005602000E9
:1036C000A83003602300FA20F8338000186023003C
:1036D0006420A433186023005F38AC3318602300E3
:1036E0000338B03318602300C630B43318602300A9
:1036F0000020B833186023003825FC339D604D4D01
:103700005A665D644C4D9A64DD619625AD001D627C
:103710004A4D9A675D62F53DFF3D9D621E25484A10
:10372000DD6618675867D9651966DA67BE23C02158
:10373000444A5B00E250444B4900635004316250FC
:10374000C4225200A350FA23E4205B000432A350A9
:103750000432A3503D493E4A3E4BD1603E49800071
:1037600019503E49E938FF3819503D490430195085
:103770003C491038D1613C4911633C4951633C4993
:1037800011603C49195019003B48F83108603B4929
:10379000D16582213A4A89005A501A0039490832C3
:1037A000D1671A003849B43211608821374A89003C
:1037B0005A501A00364988321160364ADA6408F0E5
:1037C000C3F9012008F050F970BD200014259C3089
:1037D000056020000435A03070E7200010259C30E3
:1037E000056020000335A03068E720000E259C30DE
:1037F000056020000235A03060E7C0460004FF1FCE
:103800004467FF1F3072FF1F0047FF1F4A0AFF1F58
:103810003A07000080C3C9019A02000050C30000AB
:103820006A180000280A0000204E000088130000DB
:10383000F009FF1F001F001168100000C4090000FC
:10384000DC05000040420F0010270000FD1BFF1F99
:10385000FC00FF1F0000FF1F012FFF1F2932FF1F69
:10386000C130FF1FD51FFF1FF11FFF1F9D21FF1F2D
:10387000491FFF1FC128FF1F692CFF1FD918FF1FF9
:10388000CD27FF1F3525FF1F4125FF1F491EFF1FA5
:10389000011FFF1FC11DFF1FF7B50B0CFF270122E2
:1038A000009300233C001E001D009446019089B245
:1038B00062469A401000084018413618B6B2FF2FF1
:1038C00002D1012E00D19FB2009802401A41AD18DA
:1038D000ADB2FF2C02D1012D00D19CB20133102BCF
:1038E000E6D10320012E07D1012D04D1019B240133
:1038F000E4191C700138FEBD102EFCD10238102DC9
:10390000F9D00230F7E710B5064C2378002B07D129
:103910000548FFF7F1FD0548FFF7EEFD0123237091
:1039200010BDC0460467FF1F1867FF1F0867FF1F11
:10393000F0B58BB00D0001230190102936D8FFF7A8
:10394000E2FF00231A001B48C15C01335218102B00
:10395000FAD1023B002A29D0174B184C1F680023CC
:1039600006A9E25C1600FA5C56405E540133102B47
:10397000F7D102AA08F008FA2A0002A9019808F073
:103980007BF907F0A1FF23681B18236007F09CFF59
:1039900063681B18636007F097FFA3681B18A36098
:1039A00007F092FFE3681B18E360002318000BB0D8
:1039B000F0BDC0461867FF1FA045FF1F0867FF1F27
:1039C0000223F0B50124614D614E2B70614B91B023
:1039D0001C70614F0393336800210820BB7006F010
:1039E000D3FD082006F0CAFC0023984205D0BA781F
:1039F000552A02D0332A00D09BE03360002006F025
:103A00003DFF07F011FFFFF79BFD08F0DDF91F22D6
:103A100001240021514B10AE1A70514B1C70514BB8
:103A20001970514B19689143163A0A431A60602283
:103A300019689143403A0A431A6007F04DFF07F0B6
:103A4000FBFFC120FF21494B80001A588A431A50BE
:103A5000C522920098588843BF390143995098581D
:103A6000434908408021C901014380209950995859
:103A7000C0050902090A0143995080213D484901C6
:103A800007F032FF032322003B49019400933B4897
:103A900008F002F82C223A4905A808F04DF805ACC8
:103AA00061782078023406F089FCA642F8D1354CC2
:103AB0000020012106F096FD2268334B03201A40B6
:103AC000A023DB0213432360802322689B0413435B
:103AD000236022682D4B1A4080239B0313432360ED
:103AE0002B4A2C4B934200D8012008F0FDF808F037
:103AF000E3F880232268DB0413432360287808F06E
:103B000003F9039B1878C0B208F046F907F05CFE91
:103B10002149042008F000F806F07CFE00F0B4F81B
:103B200000F0FAFD00F08CFE00F01AFA002011B04F
:103B3000F0BD00932100184A042007F01DFF8023E8
:103B4000DB059C62FFF782FC58E7C0464A0AFF1F6C
:103B500034F000400047FF1F9C64FF1F480AFF1F0E
:103B6000490AFF1F680AFF1FBCF0004000E100E0A7
:103B7000FF00FFFF0447FF1F8859FF1F0457FF1F67
:103B800068BE001114F00040FF7FF8FFFFFF9FFFA9
:103B90000080FF1F3072FF1F3B00010870B5002539
:103BA0002A492B4A2B484D6308CA1B051B0DED18EB
:103BB0008242F9D10022284B8B63284B08211A62DC
:103BC0008022274B9205DA67264BDA688A43DA604F
:103BD000254A1278012A03D09A6824490A409A603B
:103BE00000260121224C11202660DA688A43DA601F
:103BF00007F012FE112007F0C7FF8022636C934389
:103C00006364EE24E4006C431A4A200C040064232D
:103C100090420AD8FA223300D200904205D9164BBE
:103C20000A21C01807F068FFC3B2144A11201372AA
:103C3000D48007F099FF124B1B78002B04D1114B55
:103C40001021187808F0E8F870BDC0460000054063
:103C50008805054000060540FF01000000F0004017
:103C600004E100E03CF000404A0AFF1FFFDFFFFFD5
:103C700000380040B70B000030F8FFFF8464FF1FDE
:103C8000BE66FF1FBC64FF1F002210B5110011208B
:103C900008F062F810BD0000F8B5002301250826E1
:103CA000394F3A4C3B62E3681120AB43E360E36871
:103CB000B343E36007F068FF112007F0ADFD11206A
:103CC00007F08AFF402322680221134323608023E8
:103CD0006268DB02134380226360A36807201343FA
:103CE000A360A3682A4A1340A3608023A2689B01B3
:103CF00013431022A360236C93432364236C2B4350
:103D0000236480235B003B62226B224B1A402263B8
:103D1000626B1A406263A26B1A40A263E26B1340AB
:103D2000E3631D4AE3681340E36006F047FB2900A4
:103D3000072006F057FC8021184A1120536C0B43D2
:103D4000536407F0F9FFFD21154B164A89005A50BC
:103D50008023C720626B5B0313436363E3688000C7
:103D60003343E360E368104A1D43104BE560195884
:103D70001140802212020A431A50802292051A60D2
:103D80000B4B5E63F8BDC04600F000403CF00040C5
:103D9000FFFFDFFFEFFFEFFFFFFF7FFF0038004077
:103DA0000000FF1F9D3B0011FF00FFFF00E100E04E
:103DB0000000054030B503A804880B20002C0ED16C
:103DC0004968074D08784978090201430A20A94249
:103DD00005D1012120001980024B1B7A137030BDE0
:103DE000192A00008464FF1FF7B5150008AA168879
:103DF0004A680F4F14785278120222430A24BA42BA
:103E000014D10122DBB2019200962A0007F052FC85
:103E1000041E0BD1074B1B68002B07D068782A784B
:103E20000002104342425041013098472000FEBD3D
:103E3000022900000864FF1F30B501250379040042
:103E4000BFB02B4212D00A49408806F09FFF28429B
:103E50000CD06A46074B69465B8D55801380064B34
:103E600060881B7A1371002204F070F83FB030BDF7
:103E70000064FF1F3043FF1F8464FF1F10B5054916
:103E8000054806F039FF0421044A054806F0F6FE0D
:103E900010BDC0460064FF1FFFFF000094BE00116C
:103EA0003043FF1F10B5024804F0D2FE10BDC046DB
:103EB000393E0011062310B5837010330371443B63
:103EC00043712A3383714433C371002302220121D9
:103ED00003720E4B027041701C8881724472197A11
:103EE0000273C1729A784273DA7882730322C273C2
:103EF0001A7902745A7942740C2282749A79C274C3
:103F0000DB7903751123C370152010BD8464FF1F76
:103F100010B5122007F0D8FD104B122200211860B6
:103F200007F092FF002007F05FFF012007F0FCFE82
:103F3000022004F031F9032006F046F9042003F0D2
:103F40006FFB052004F03CF8062001F03DFA072045
:103F500006F074FE082001F017F810BD0C64FF1F76
:103F600010B507F0D1FD012007F0FEFE07F044FC7C
:103F7000002010BD094B10B50400984205D001295E
:103F800004D12000064906F0B7FE10BD0229FCD17D
:103F9000013904F01BFE0028F3D0F6E7FEFF000015
:103FA0003264FF1F70B50D7A100004AA2C00168829
:103FB00010221440154220D1002E20D10A78022A66
:103FC00018D14A68517815780E4A0902294391425E
:103FD00005D00D4A914209D01C800A2404E0142225
:103FE0000A491A8007F0A8FD200070BD0C2208497C
:103FF0001A80F7E71C800124F6E70824F4E70B2475
:10400000F2E7C046F3FF0000F4FF00008445FF1F05
:104010006CBF001110B504000749084806F06CFE9B
:10402000074804F055FD0020E40704D50721054AA0
:10403000054806F023FE10BD3264FF1FFFFF00009D
:10404000753F0011D4BE00117443FF1F00B50C4B27
:10405000BFB01A780B4901A800F0ACFC6B4680B2E7
:104060005880002809D06A46074B69461B88138090
:10407000064B0022188803F069FF3FB000BDC04620
:104080001064FF1F1164FF1FCE43FF1FD844FF1FA2
:1040900000B50C4BBFB01A780B4901A801F09CFE8B
:1040A0006B4680B25880002809D06A46074B6946A3
:1040B0005B8D1380064B0022188803F047FF3FB04A
:1040C00000BDC0463A64FF1F3B64FF1F7443FF1FDF
:1040D000D844FF1FF7B50E00377A1C0008AB11005B
:1040E0003D001A8820231D401F423CD13378022B0B
:1040F0003BD173681F785B781B023B431E4FBB426A
:1041000008D01E4FBB4214D01D4DAB4221D00A2512
:104110002800FEBD002A2AD1142C2AD82200F068DB
:1041200007F00AFD174B1C70012CF1D9FFF7B0FF07
:10413000EEE7002A1BD1202C1BD82200F06807F0E4
:10414000FBFC114B04211C70104B187807F064FE27
:10415000DEE7E3B20124009201940A00310007F087
:10416000A9FA0500D4E70825D2E70125D0E70B25F9
:10417000CEE70D25CCE7C046F3FF0000F4FF0000BA
:10418000022900003A64FF1F1064FF1FBC64FF1F78
:10419000332310B5040003700A220749013007F0E9
:1041A000CBFC064B0F201B681A0AE37222731A0C11
:1041B0001B0E6273A37310BD8464FF1FAC64FF1FEA
:1041C00030B5012503790400BFB02B4213D00B4951
:1041D000408806F0DBFD28420DD06A46084B01A856
:1041E0001B881380FFF7D4FF6B4658800022694676
:1041F000608803F0ABFE3FB030BDC0463264FF1FA5
:10420000CE43FF1F10B5024804F022FD10BDC0468A
:10421000C141001170B5160004AA148805AA1578CA
:104220004A685078117800022A4A08438018052805
:104230004BD807F011FE03131E29343F0720032C2F
:104240000BD80422121BAA4200D92A0022491A8044
:104250003000091907F070FC002070BD0720112CF8
:10426000FBD81222121BAA4200D92A001B491A802D
:10427000EEE707200E2CF0D80F22121BAA4200D91D
:104280002A0017491A80E3E70720032CE5D8042207
:10429000121BAA4200D92A0012491A80D8E7072027
:1042A000032CDAD80422121BAA4200D92A000E4994
:1042B0001A80CDE70720032CCFD80422121BAA4274
:1042C00000D92A0009491A80C2E700220A201A8070
:1042D000C3E7C046DCD5FFFF1FBF00115864FF1FB6
:1042E0000FBF00110ABF001105BF001100BF001170
:1042F00010B50D21024A034806F0C0FC10BDC046AF
:10430000F4BE0011E443FF1FF0B50024274E85B032
:104310003000B47100F0E2F8254D264BEA89297C83
:104320009A422FD10423300003AA00F057F9040069
:10433000300000F011F90123B371002C34D16B4629
:1043400099892B68C9BA4B4329891B4A1B145B18EE
:1043500053806B46D9896B6849BA89B24B436989E6
:104360001B0C5B181548191C1BB2834200DD011C95
:104370000B0400D5002113889180013313802000A5
:1043800005B0F0BD0227220003AB3000009700F01B
:10439000F7F80E230400297C0122300000976B44BB
:1043A00000F0EEF80443C3E71C00E8E7BC44FF1F3D
:1043B0006C64FF1F830500008464FF1F0F2700004B
:1043C00073B5234E300000F089F8224D07236A466A
:1043D0003000297C00F002F904003000002C33D1B9
:1043E0006B461B787F2B2FD800F0B6F86B46D87839
:1043F000F02302041B031A406B469B8816495BBAE4
:104400009BB21A432B68000953432A891B0C9B1843
:104410004B806B465A789B7812031B011A436B68DA
:10442000024353436A891B0C9B180C481A1C1BB28D
:10443000834200DD021C130400D500220B888A8011
:1044400001330B80200076BD00F086F80124F9E7E7
:10445000BC44FF1F6C64FF1F8464FF1F0F27000014
:1044600070B5114C237C002B0FD0382B0ED10F4D83
:10447000280000F033F8CC23AC222800217C9B01DB
:1044800000F0F4F8280000F067F870BD084BE289EE
:104490009A42FAD1054D280000F020F800222800A9
:1044A000217C00F0C5F8EDE76C64FF1FBC44FF1FE2
:1044B0008305000010B5084B1A7C002A09D05B69FF
:1044C000002B06D09847041E01D0FEF799FD20006E
:1044D00010BD0124F9E7C0466C64FF1F70B5C179B7
:1044E00005000C00631E9C411A4BE402E4184900CD
:1044F0000460C9B2007906F0ABF8E979687949003F
:104500000131C9B206F0A4F8E8790930C0B207F069
:1045100063FB0023E36661332360AA795B3B002AD7
:104520000ED022689A43023B134323600A23E361BF
:104530000733236200232363A3630133E36370BD66
:1045400022689A43022313432360462363610633A0
:10455000A361EFE70050004070B500250400036838
:10456000DD66C0790930C0B207F00EFB2900207962
:1045700006F00AF82900607906F006F870BD000020
:10458000F8B51E0006AB1D78002304681700E3662B
:10459000616007F091F901238022E3662B00276117
:1045A0005200013B08D207F03FFA08200A4A11687E
:1045B000002D03D12800F8BD2261F2E7236F0342EA
:1045C00003D02369013D3370013613685B1A032B56
:1045D000EED90125EEE7C0466008FF1F70B51C004C
:1045E000002305681600EB66696007F065F9012392
:1045F0008022EB6623005200013B08D207F014FA38
:1046000008200A4A1168002C03D1200070BD2A61DD
:10461000F2E72B6F034203D02B69013C3370013664
:1046200013685B1A032BEED90124EEE76008FF1F25
:10463000002370B504681500E366616007F03CF97B
:104640000123E366256107F0EFF98020064A800028
:104650001168636B034205D113685B1A032BF8D909
:10466000012070BD0020FCE76008FF1F70B51D0031
:10467000002304681600E366616007F01DF901235A
:10468000E36626610F33626B1A42FCD02B0A23616A
:104690001023626B1A42FCD0EDB2256107F0C4F919
:1046A0008020074A80001168636B034205D11368BC
:1046B0005B1A032BF8D9012070BD0020FCE7C0462F
:1046C0006008FF1F70B51E00002305681400EB662C
:1046D000696007F0F1F80123A619EB660F33B442C5
:1046E0000ED107F0A1F980200A4A800011686B6B97
:1046F00003420CD113685B1A032BF8D9012070BD5B
:1047000021782961696B1942FCD00134E7E7002068
:10471000F5E7C0466008FF1F10B5084CE368002BA2
:1047200008D1074B1B685B045B0C0A336360054BC5
:104730001B68236007F050F8A06010BDAC64FF1F39
:10474000C8F00040CCF0004010B507F0B5F80F4BB2
:10475000996A9A6A8A42FBD10D4C6268A0688A18ED
:10476000121A531E884200D31300A1602168DA0B8D
:1047700052185B0407495B0C636022600B60064BB8
:104780001A6007F051F9206810BDC04600F00040E3
:10479000AC64FF1FC8F00040CCF0004070B51F4C67
:1047A00023793F2B01D93F2323711D4B22791A70A6
:1047B0001878C0B207F040FB18231A491A4A0B8038
:1047C0001A4913800B805380A379194980200B80EC
:1047D0000C21938001334B43164D191C0001834279
:1047E00000D9011C2980D1806379002B11D10133BC
:1047F0006371237A012B01D8022323726279237A11
:104800000D4853430A21584307F076F90B4D2860B1
:1048100070BDA02BEDD9A023EAE7C046A064FF1F1E
:10482000480AFF1FD644FF1FAC46FF1FD444FF1F9A
:10483000D244FF1FD044FF1F710200009064FF1F8D
:10484000F8B513210020FEF7C9FD114C011E114DD2
:1048500009D10C22104BC1CBC1C4280007F0F4FAD7
:10486000FFF79CFFF8BD0C2220000C49FEF78AFDE3
:104870000C2802D0084B43CB43C40C222800084923
:10488000FEF780FD0C28EBD00C220021E5E7C046A6
:10489000A064FF1F6C64FF1F60BF0011FC0C0000D0
:1048A000F50C0000F0B51D4C8022A54404008820C2
:1048B00069465201400507F0A7F8902212016A44A8
:1048C0001300200032C832C316C816C38023144C0C
:1048D000144FA6689B033343A3603B6007F01CF8AA
:1048E0008823A0685B05C01807F026F800258823F8
:1048F00029008022A0685B05C01840196944520055
:1049000007F03AF980230135FF355B019D42EED176
:10491000A6603E60044B9D44F0BDC046FCEFFFFF27
:104920001C46FF1F9808FF1F04100000F0B504008C
:1049300087B0002825D0684607F0A6F91B4C02284E
:1049400006D106226946200007F046F8002816D056
:104950006946002301250F262F00E25C0133100970
:104960001030874038002F00324097403A00024311
:104970004A610439062BEFD16846FFF793FF07B071
:10498000F0BD182269460A4807F03EF86A46A300BF
:10499000D358013305D01822FF21684607F054FA96
:1049A000EAE70134062CF1D1E9E7C0466509FF1FAB
:1049B00000090011F0B5002504000E0085B0AA42E0
:1049C00000D186E04B1C087801934B7889783779C1
:1049D00009021943F3783F061B040B431F43039757
:1049E00020706570252800D196E033D8112813D89F
:1049F00007F012F869001F011F011F011F01AA0023
:104A0000B800B1001F011F011F011F011F011F017D
:104A10001F011F01FF001901232800D1D8E0DB2866
:104A200000D028E1042A00D8ACE01025052A05D0E2
:104A3000551F2A003800711D07F07EF8052231004D
:104A4000200007F079F82A003900601D07F074F89B
:104A500005353EE0562859D010D8332800D19DE0C6
:104A6000552839D02628DAD1984B2900132218006E
:104A70001D0007F0E9F9FEF7C3FA5CE0712800D1E8
:104A800077E0722800D180E0602800D18BE0DC283C
:104A9000C5D1022A00D875E07378BFB26370B378CD
:104AA000A370032A05D0033A390092B2F01CFEF736
:104AB000A3FB10223900E01CFEF764FCC51C002893
:104AC00007DA60705CE00C222000814907F034F8BE
:104AD0000C25280005B0F0BD013A7E4D0C2A13D8F4
:104AE000002A0AD02800019907F026F8FFF756FEA1
:104AF0000C2228007849FEF77FFB29000C22601C5D
:104B000007F01AF80D25E4E70C22EBE7714D734B23
:104B10002A0043CB43C2E9E7013A6C4D0C2A11D875
:104B2000002A08D00199280007F006F80C22280076
:104B30006B49FEF761FB29001322601C06F0FCFFA5
:104B40001425C6E70C22EDE705226649601C06F035
:104B5000F3FF0625BDE712226349601C06F0ECFF57
:104B60001325B6E708226149601C06F0E5FF092518
:104B7000AFE77178F72905D85D4B188801F088FDFB
:104B80000225A6E7FF236370FAE75A4B012A03D0F8
:104B900072785A706270F3E75B78F4E72000FFF7F1
:104BA000F7FA050095E7013A534D062A0ED8002A78
:104BB00005D00199280006F0BFFF01F03FF8290059
:104BC0000622601C06F0B8FF072582E70622F0E700
:104BD000042A04D9494D2F6006F0FEFDA860FFF7B6
:104BE000B3FD0422039003A9601C06F0A5FF052570
:104BF0006FE7434D062AE2D906222800019906F004
:104C0000EBFE0028DBD006220199280006F094FF75
:104C100006223C492800FEF7EFFA0123354A517875
:104C20000B435370CBE7012AACD07078FFF77EFEC0
:104C3000A6E7012800D0F2E6931E334F1A2B04D8C2
:104C40007378002B09D100F013F9304B39001D782F
:104C5000601C6A1E06F070FF3BE7551E2A00019992
:104C6000380006F069FF2A49AAB23800FEF7C4FAF4
:104C700000F034F9E9E7DA281CD1042A82D9082A9D
:104C800015D9B37972791B021343F27912041A43CE
:104C9000337A1B0613433B603B680522310020003A
:104CA000039306F049FF0422601D03A95DE7FE237C
:104CB0006370F1E7DE2800D064E7511E012A01D1BC
:104CC000002506E7019800F09FFFF9E76C64FF1FDD
:104CD0006CBF0011A064FF1FFC0C000060BF00113E
:104CE000F50C00007864FF1F5864FF1F2046FF1F6B
:104CF000D844FF1F9C64FF1F7545FF1FAC64FF1F56
:104D00006509FF1FADAC00009D66FF1F9B66FF1F7E
:104D1000AEDE000070477047020010B5094B0A3242
:104D2000094C92B2DA815A8298811882207802F076
:104D300015FB0422054B012120781A7007F06CF84E
:104D400010BDC046AA45FF1FE666FF1FE566FF1FB0
:104D5000013870B5042809D807F07EF8030928083F
:104D60001200234B0221187807F056F870BD204B33
:104D70000821187806F0E8FD00221E4B1A72F5E7AC
:104D8000802200241B4B1A4D52001A8108211A68F8
:104D90002878DC7206F018FF2100287806F0E4FD80
:104DA000012000F069FE00F049FFDFE7104B082109
:104DB000187806F0C9FD1048FFF77CF80F4B104A31
:104DC0009B79002093800F4A13808022094B520068
:104DD000D8721A8100F050FE00F030FF0A4B5B7869
:104DE000002BC3D0094A136006F0B6FEBEE7C046EA
:104DF000BC64FF1F9064FF1FE144FF1FA064FF1FFE
:104E0000AC46FF1FD244FF1F9C64FF1F34F00040DC
:104E100010B501290BD1082809D1054B1B78002BAF
:104E200005D02622034B04485A72FFF775FF10BDC8
:104E3000BE66FF1F9064FF1FC40900000300F0B5A9
:104E40000A4D8E18B14202D152008018F0BD0C7884
:104E50002F6824093C5D0F271C700C7801313C4001
:104E60002F683C5D5C700233ECE7C046CC44FF1F0A
:104E70000D22114B10B51A700C23104C10492370E1
:104E8000093A033B0F48637006F056FE2D230122BA
:104E90000D490E48A371FFF7D1FF01220C49FFF71E
:104EA000CDFF01220B49FFF7C9FF00220A4910007C
:104EB000FEF7A2F910BDC046BA66FF1F9B66FF1F32
:104EC0001FBF00119D66FF1F6709FF1FA266FF1F1E
:104ED0006609FF1F6509FF1FAEDE000070B5124CAA
:104EE000132220001149FEF74DFA114D002817DD5D
:104EF000AB78002B14D0431C2B7009236B7000235C
:104F000000190370287829000130C0B206F004FFB0
:104F1000297822000139C9B2002005F0CDFD70BD0D
:104F2000FFF7A6FFEEE7C0469D66FF1FAEDE00005E
:104F30009B66FF1F10B5114B1A781870002A0ED00F
:104F400000280BD10E4B1A78062A07D85423D340D9
:104F5000DB0703D50B4B187802F000FA10BD0028D0
:104F6000FCD0074B1B78012B02D0033B022BF5D85A
:104F7000044B0121187806F04FFFEFE7BE66FF1FD4
:104F8000E566FF1FE666FF1F70B5514E514A524954
:104F90003070082005F01CFC0121022005F022FBE6
:104FA000022005F003FC0121002005F01BFB00207E
:104FB00005F0FCFB00F0ACFEFEF722F806F03CFE2C
:104FC000032246494648FFF739FF2D2403000422F7
:104FD0001C7044490130FFF731FF30230470424D0B
:104FE000424C437083702E3B062220004049EB87E1
:104FF000FEF7C8F9062813D0200006F045FE022867
:1050000009D00321200006F047FC8D23E3706E3B9E
:10501000237119336371062220003549FEF7ECF83D
:10502000344B1B68FC335C64FFF758FF0020FFF72C
:1050300081FF314C314A0121314B1278207802F046
:105040004FF9304A304B12780021207802F048F9AD
:1050500001222E4B1A702E4B9B78552B31D12D4BA4
:105060003B325A722C4B2D4AAB81EA812B826A82E9
:105070002021307806F0E8FD0120404205F068FD6F
:105080000120404205F004FEFFF732F9FEF7F6FE7C
:1050900000F0A6FC01204042FEF7BCFF012006F014
:1050A000B3FEF72001F0D8FA0121307806F0B4FE03
:1050B000307802F0AFFA1A4806F086FCFEF7ECFDF5
:1050C00070BD6422174B5B7953431A000A32CBE759
:1050D000BC64FF1F154D0011114E00112046FF1F2B
:1050E0005864FF1F7864FF1FAA45FF1F6509FF1F53
:1050F000ADAC00004467FF1FE666FF1F0045FF1FC1
:10510000E144FF1FBA66FF1F9B66FF1F8C66FF1FEF
:105110009C64FF1F9064FF1FC4090000CE090000BB
:10512000BE64FF1FA064FF1FF8B50A0020230D0016
:105130001A40194257D0574B1B78002B50D0FFF71D
:1051400003FB554B554C564E99686268737A8A1A20
:10515000DB039A4202D36160FEF79EFD327A217A28
:10516000531EDBB2994205D1FFF77AF9002000F017
:105170009BFD0FE09142F9D300232372FFF79AF9C8
:10518000012000F091FD474F3800FEF793FE3900F3
:1051900006F012FE637A002B1FD0013BDBB2637274
:1051A000002B1AD1404B9B78552B01D106F0D4FC33
:1051B000E37A002B0CD000233C4A3A4FE372138869
:1051C000380001331380FEF775FE390006F0F4FD58
:1051D000642370795843FFF79FFD237A01332372CC
:1051E00020206840F8BD0BB2002B0ADA304B18784B
:1051F00006F08AFB002801D006F076FC8020000231
:10520000EFE70224214206D0244B01201A72FFF757
:1052100091FE2000E5E70B071ED5FFF795FA1E4B20
:105220001E491F4C98684A68637A821ADB039A42C7
:1052300002D34860FEF730FDFFF73CF9FFF710F9A5
:10524000012000F031FD00F0E5FB2368DB0701D50C
:10525000FEF7D8FF0820C4E71024214206D00D4BEA
:105260001B78002BD5D1FEF71DFED2E70124214289
:1052700007D0104800F06CF806F0BEFD00F0FAFC14
:10528000C7E70424080020402142ABD0FEF7DEFE31
:10529000BFE7C046BE66FF1FAC64FF1F9064FF1FE0
:1052A000A064FF1FE144FF1F9C64FF1F8464FF1F75
:1052B000BC64FF1FC444FF1FF0B51B4B1B4F1B8872
:1052C0003A8804001A4E1B4D85B09A420DD8328898
:1052D0009A420AD3184B1A882B889A4205D1174A4A
:1052E000174B12881B889A421BD0052001F00AFA3E
:1052F0003B8802AA13803388019053802B88114D7C
:1053000093800F4B02A91B88D3800F4B2A781888F3
:1053100002F026FF0D4B08212878019A1C7006F038
:105320009BFA05B0F0BDC0468A66FF1FD644FF1F3A
:10533000D444FF1FD244FF1F8866FF1F8666FF1FED
:10534000D044FF1FE666FF1FD844FF1F8466FF1F7F
:1053500013B50C4B1C78002C11D1002801D00A4B3E
:1053600018600A4A0A4B11780A4A10780A4A0192D0
:105370000A4A0092002205F097FA200016BD112477
:10538000FBE7C046E566FF1F8066FF1FE466FF1F60
:10539000D466FF1FE666FF1FC066FF1FC466FF1FBF
:1053A00010B5064B12201B78052B06D1044B132297
:1053B0001988044B187801F081FB10BDE566FF1FCA
:1053C000D844FF1FE666FF1F10B500240122114BD1
:1053D00052421870104B1C70104B1A8002F01AF9D0
:1053E00004220F4B21001A700E480C3206F034FBD9
:1053F000102221000C4806F02FFB07220B4B1C60EB
:105400000B4B1C700B4B1C700B4B1A700B4B1C7016
:1054100010BDC046E666FF1FE566FF1FD844FF1FAC
:10542000E466FF1FD466FF1FC466FF1FC066FF1F30
:105430009A66FF1F9966FF1FDA44FF1F9866FF1FD9
:10544000F8B5174C0600257806A814240078052D19
:1054500023D1B41F134FA5B21824BD421DD88D1FF0
:10546000ADB2BD4219D8FA256D00AA4215D21D0071
:105470000D4F0A3DADB2BD420FD80C4C26800C4CEE
:1054800021800C4900240A800B4A1380FFF714FF87
:105490000A4B0421187806F057FA2000F8BDC046E0
:1054A000E566FF1F790C0000750C0000D644FF1F55
:1054B000D444FF1FD244FF1FD044FF1FE666FF1FE6
:1054C000F0B50BB20D0089B0002B00DB70E1A44EEB
:1054D000307806F019FA041E50D00378A22B00D1C0
:1054E00022E1D02B1AD0912B45D143780E2B42D1FB
:1054F0009C4B82889A423ED19B4A83681278052A47
:1055000039D1032018567F2835D0984B1B68002BC3
:1055100031D05B68002B2ED098472CE0807807288C
:1055200029D806F099FC0428183F3F74A8D863785E
:10553000002B0CD101218C4B19708D4B1A78002A4D
:105540005BD08C4B307801F0CBFE002855D0072281
:10555000854B1A7051E061780029F8D1E378002B6F
:1055600011D0854A854B1278307801F0B9FE607011
:105570006378002BEBD1200006F0B6FA8020000201
:10558000684009B0F0BD784B1B78022BF3D00121A5
:10559000307806F0C9F90028EAD10121307806F008
:1055A0003BFCE5E76378002BD1D16F4F032807D18F
:1055B0003B78052B02D101333B701EE00223FBE751
:1055C0006F4B1A886F4B0293002A0BD01B78002B6D
:1055D00003D00121307806F03FF93B78062B04D147
:1055E000013BE9E7029B1A70F7E7042B41D1012147
:1055F000029B3078197006F00FFC5C4B1B68002B87
:10560000B9D01B68002BB6D0574A107884E763786E
:10561000554F002B27D10622211D5B4806F08CFA3E
:1056200062895A4B5A491A80A2895A4B1A80E389D7
:105630000B800521397058490A80584A1380228A04
:10564000574B1A80574B1B78012B09D11F2001F0B3
:1056500059F8FA22920042430421307806F0FCF80F
:105660000022484B75E7312B00D070E70022454BF4
:105670001A700323A0E706220021434806F0ECF944
:105680000023454A04211380444A30781380444A59
:10569000138006F059F90821307806F055F9A379FE
:1056A000083B5A425341304A03331370304B1B7846
:1056B000002B06D0334B30781A78002A06D001F040
:1056C0004DFE0122314B52421A8096E7012119709A
:1056D00006F0A2FBF5E70821307806F035F963788B
:1056E000002B00D047E72C4B2D4F0293E388029A02
:1056F00004211380294B307803932389039A138064
:1057000063893B8006F010F9002800D033E7264B70
:105710001B68002B00D12EE7039902983A8809886C
:1057200000881B68984726E74379132B00D022E7AF
:105730000389012B0AD11D4B1B78022B06D10821AE
:10574000307806F001F9FFF72BFE14E7052000F092
:10575000D9FF08210200307806F07EF80BE7C0463A
:10576000E666FF1F05140000E566FF1F8066FF1F49
:105770000045FF1FE144FF1FBA66FF1F9B66FF1F26
:10578000BC66FF1FBE66FF1F8D66FF1FD844FF1F4C
:105790009466FF1F9666FF1F8A66FF1F8866FF1FBD
:1057A0008666FF1F8C66FF1F7C66FF1F8466FF1FD7
:1057B0008020C001014200D0E2E6CB0731D5324B58
:1057C0001B78002B1DD0314E05AC3378052B1AD138
:1057D000023B23702E4B21001B7823722D4B1B782C
:1057E00063722D4B187801F01FFD002809D00720A7
:1057F0002A4B30701B68002B03D01B68002B00D095
:1058000098470120BCE60E20254B06221B7825492F
:105810002370254B1B78637002ABC01806F08CF91F
:10582000D8E7022308001840194209D0174B1B780B
:10583000052B03D11D4B188806F0B6F902209FE610
:105840000424214203D0FFF737FD200098E6082307
:1058500008001840194200D193E6154B1C78012C22
:1058600003D0022C0DD008208AE6124B124A1349AD
:1058700013481B881288098800880094FFF7E0FD10
:10588000F1E7FFF78DFDEEE7BE66FF1FE566FF1F40
:10589000DA44FF1F9866FF1FE666FF1F8066FF1F42
:1058A0009A66FF1FDB44FF1F9966FF1FD844FF1F46
:1058B0008466FF1FD044FF1FD244FF1FD444FF1F44
:1058C000D644FF1F10B502A804880B20002C10D16D
:1058D000496808784978090201430C48814209D196
:1058E000022119800A4B59881170DB7800205BB2C5
:1058F000537010BD074C0A20A142FAD10221198031
:10590000034B998811705B79F0E7C0466E2A00005E
:105910008464FF1F6F2A0000F7B5150008AA1688D7
:105920004A680F4F14785278120222430A24BA426E
:1059300014D10122DBB2019200962A0005F0BAFED2
:10594000041E0BD1074B1B68002B07D068782A7800
:105950000002104342425041013098472000FEBDF2
:1059600002290000F866FF1F30B501250379040005
:10597000BFB02B4227D01549408805F007FA2842CE
:105980000DD06A46124B69465B8D1380022353800B
:10599000104B5B8893806088002202F0D7FA0E4992
:1059A000608805F0F3F9C0070DD56A460B4B6946D0
:1059B0001B88138002235380064B9B88938060884A
:1059C000002202F0C3FA3FB030BDC046F066FF1FB0
:1059D0000445FF1F8464FF1FE866FF1F5E45FF1F2D
:1059E00010B5074C0749200005F086F9200006494C
:1059F00005F082F90721054A054805F03FF910BD79
:105A0000FFFF0000F066FF1FE866FF1FECBF0011FC
:105A10000445FF1F10B5024803F01AF910BDC04637
:105A20006959001170B55F25082607498400CA78B6
:105A30008B7840012A40B3433440A84323430243B8
:105A40008B70CA7070BDC0467545FF1F010043B220
:105A500004205A0002409B000C3003401A431523D7
:105A600010B5044CE0789843143B0B4018430243B4
:105A7000E27010BD7545FF1F10B5054B082419795C
:105A80000A00A243002801D022000A431A7110BD67
:105A90007545FF1F10B5054B4024D9780A00A24375
:105AA000002801D022000A43DA7010BD7545FF1F9F
:105AB0000821F8B5324D334BAE7804000E40AE707D
:105AC000984204DD67232B70473B6B70F8BD2E4B6B
:105AD000984203DAE0232B703A3BF6E700232B7061
:105AE0006B7083B21A0029485F3292B2284F82420B
:105AF0002CD9002C03DA5B421CB204232B70053432
:105B000020B20A2105F0F8FF04B2FA239B009C4260
:105B100032DB08232A7813432B706421200005F020
:105B2000EBFF0A2100B205F05FFF09B22A787B5C27
:105B300013432B700A21200005F0DEFF0A2100B27A
:105B400005F052FF09B27B5C6A780AE06970002CAC
:105B5000DBDA5B421CB204232B70F3226B78092C36
:105B6000E8DC13436B700A21200005F03DFF09B209
:105B70007B5C1E43AE70A9E7632CCEDCEDE7C0462C
:105B80007545FF1F1B4E00001DFCFFFF2A0800008B
:105B900016C000110823F7B5194FCD003E79040057
:105BA0001E403E71EDB2632806DD5F3333433B7127
:105BB00020231D437D71F7BD0300093305DA20233F
:105BC0005B4233433B71A623F3E70E4B019300285E
:105BD0000BDA0423444224B23B710A21200005F071
:105BE00003FF019B09B25B5CE3E70928F5DD0A21AD
:105BF00005F082FF019B00B21B5C1E433E71ECE787
:105C00007545FF1F16C00011F8B50A4F05003B7817
:105C10000E00002B0CD0084C2000FEF75FFC330078
:105C20002A0020003978FEF74DFD2000FEF794FC95
:105C3000F8BDC0460367FF1F7C45FF1F70B50A4EC5
:105C40000A4D06223100280005F0C6FE002809D0C2
:105C5000074C31000622280005F06EFF07212000C6
:105C6000FFF7D2FF70BDC0467545FF1FFD66FF1FE1
:105C7000FC66FF1FE622402110B50A4B1A70403A1D
:105C80005A703E329A70DA780A40DA70082219792E
:105C90001140053A0A431A7197225A71FFF7CEFF55
:105CA00010BDC0467545FF1F10B500282AD0164C00
:105CB0000A210223E05E05F01FFF00B2FFF7F8FEA5
:105CC0000423E05E642105F017FF012100B2FFF715
:105CD00061FF237A0024132220009A426041C0B25F
:105CE000FFF7D8FE0320FFF79DFE2000FFF7AEFE72
:105CF000064B1878053843425841C0B2FFF7BCFE46
:105D0000FFF79CFF10BDC0468464FF1FE566FF1FC0
:105D100070B500250A4C2000A571FEF7DFFB1023AB
:105D20003E212000074AFEF7CDFCA84200D13E35B7
:105D3000054B20001D70FEF70FFC0123A37170BD01
:105D40007C45FF1F06C000110367FF1F0200F0B56E
:105D500001270A480A4E51188B1A002B00DCF0BDAF
:105D6000082415784308684038404000805B013CB7
:105D700058406D08002CF5D10132EDE7FFFF00001F
:105D800026C00011F0B500250F269D4200DBF0BDB6
:105D90004C5D070944403440A400A05801357840C8
:105DA000F3E70000F0B589B06A460D000B000F273D
:105DB000110010351C780133260024093E4016706E
:105DC00054700232AB42F5D12023024AFFF7DAFFCA
:105DD00009B0F0BD2CC00011F0B54E780B7889B039
:105DE00036020C00170001901E43012A61D9954B21
:105DF0009E4200D877E001339E421CD1062A17D17B
:105E0000CA788B7812021A430B791B0413434A7920
:105E100012061A438C4B5A6100221A705A808B4A20
:105E20005A608B4A9A608B4ADA60002009B0F0BD54
:105E300088225205EEE7884B9E423CD182498B78FE
:105E4000002B00D0F6E00C2A31D10F22A378934327
:105E5000E278120213432279120413436279120684
:105E600013434B60E279A07912020243207A0004C6
:105E70001043627A12060243CA60E27AA07A1202E2
:105E8000024376484A81834208D804236E4914228B
:105E900001980B7005F050FE1420C7E71201D218CC
:105EA00089235B059A42F0D801238B70BDE7022A53
:105EB000FAD00523EAE76A4A01239642E6D1FFF7C2
:105EC0006FFA052F0CD9E378A2781B0213432279CD
:105ED00012041A4363791B061343624A0393136047
:105EE00005F03AFEA1E7584D2B78002B9DD1AB78F9
:105EF000002B00D1A0E02B8901339BB20093B34269
:105F000000D091E0132AD4D9CF7C8B7C3F021221A0
:105F100020001F43FFF71AFF874200D08EE0002EBB
:105F20003DD1E378A2781B0213432279E968120479
:105F30001A4363791B06134303930A228B4212D13F
:105F4000FF23A370E370237163716B89002B09D168
:105F5000E37B227C1B0212041343A27B13431B0925
:105F600001336B8100226B89002B8ED0002A67D110
:105F7000686837013818000B6B690003039098427A
:105F800005D9686105F0D8FCEB780133EB706868DF
:105F90001022A11C381805F0EFFD2E8145E76F890E
:105FA000009A7B1E9BB293423AD1E278A378120208
:105FB0001A43237905A81B04134362796C681206FF
:105FC0001A43EB6800920392211D0C22049305F002
:105FD000B3FD0120260004A940421036FFF7E2FE7F
:105FE000013F012F17D1009A0B232861824200D074
:105FF0004CE704221C49200005F0BEFD042203A941
:10600000686805F001FDE968039AFF23914200D119
:106010003CE7F73B3AE73100FFF7C4FE1036DFE715
:106020000923B742A4D831E7009BB34200D9FCE66C
:1060300007232BE7022329E7032327E7062325E786
:106040000A2323E7FFFE00008445FF1F0000011123
:10605000FFFF00005048593601FF0000FFFF00110C
:1060600002FF000034F000409045FF1F10B5034CC4
:106070000B000122210000F06BFA10BD2D6200110F
:106080000B8870B506000D000224162B11D92B00C9
:106090000322094900F05CFA041E0AD1074B2A8842
:1060A0001B88191C934200D9111C300089B200F0E2
:1060B000EFFA200070BDC046596200115E67FF1FF5
:1060C00010B54A780400013A0B000220012A07D8D3
:1060D0000A78002A04D005222000024900F038FA8C
:1060E00010BDC046876200110A7810B50B0004008D
:1060F0000220002A04D007222000024900F028FADA
:1061000010BDC046336300110A7810B50B000400BF
:106110000220002A04D009222000024900F018FAC7
:1061200010BDC0469963001110B5034C0B000B2243
:10613000210000F00DFA10BDC963001110B5034C29
:106140000B000D22210000F003FA10BD3B6400118A
:1061500010B5034C0B000F22210000F0F9F910BD1F
:10616000956400110A7810B50B0004000220002A83
:1061700004D011222000024900F0EAF910BDC04607
:10618000A5640011002310B51322190000F0E0F9F6
:1061900010BD000010B5034C0B001722210000F0C9
:1061A000D7F910BDF7640011002310B519221900AA
:1061B00000F0CEF910BD000010B5034C0B001B22FF
:1061C000210000F0C5F910BD31650011F7B58489D3
:1061D0000D0006000121002C22D000238268D35636
:1061E0001778002B1EDA0C2C1AD90C3CA4B2131908
:1061F00040880093230002F086FE431E9841013040
:106200007B06DB0F6B703F23013C1F40A4B228705C
:10621000AF70AC80002C07D0B3680133AB600021B5
:106220000800FEBD0020EBE7AC60F8E70B780370D8
:106230004B8843704B881B0A83700B79C370042012
:1062400070470420022B06D10020537811781B02DE
:10625000009A0B43138070470B8803700B881B0A4E
:106260004370022070470420009983420AD153787A
:1062700010781B0203430B80D37890781B020343F2
:1062800000204B807047F8B50D004B7801240021A9
:10629000461C03702B788B4201D82000F8BD6B7828
:1062A000B01C4F1C012B10D1890069184B880222A9
:1062B00033704B88B9001B0A7370691805F0DCFC59
:1062C00004360434A4B2F9B2E4E7122359436B183C
:1062D0005A88043132705B8810221B0A7370691867
:1062E00005F0CAFC12361234ECE770B5049D1400B8
:1062F0001E00052B01D8042070BD637812781B02A4
:1063000013432B80E378A2781B02134302226B8095
:106310002A71211D681D063E05F0AEFCB2B22A812D
:10632000F02AE8D82800A11D0A3005F0A5FC0020BD
:10633000E2E7002310B50A789A4201D8900010BD18
:106340009A008A185488013304705488DBB2240AF6
:106350004470948884709288120AC2700430EAE70C
:1063600010B51100029C062B04D004201022142B1F
:1063700001D010BD022222714B7808781B02034322
:106380002380CB7888781B02034363800431601D2F
:1063900005F072FC0020ECE710B50C788B78043126
:1063A0005C43E4B203702200013005F065FC601C20
:1063B00010BD0420022B06D10020537811781B0257
:1063C000009A0B431380704710B50C000A88023105
:1063D00005F052FC208810BD70B504000D00049833
:1063E0001100012B01D8042070BD167852781202DA
:1063F000324302800200F83255701470E825002CF8
:1064000000D10C35023B9AB24280AA42EBD802314D
:10641000043005F031FC0020E6E7042000998342B7
:106420000AD1537810781B0203430B80D3789078FD
:106430001B02034300204B80704710B50C000A88F4
:10644000023105F019FC208810BD000070B5012153
:106450001E000420049C0E400B4218D1CB40DDB23C
:106460008D4214D90A49DBB2098899420FD323001F
:10647000F6331D703300580011184978165C090274
:10648000314301332152D9B28D42F4D8002070BD7E
:10649000A445FF1F10B50C000A88023105F0ECFB83
:1064A000208810BD10B50C788B7804315C43E4B2C1
:1064B00003702200013005F0DFFB601C10BD10B539
:1064C00011000298032B01D8042010BD14785278D3
:1064D000043B120222430280CA788C7812022243C3
:1064E00042809AB28280F22AEED80431063005F05A
:1064F000C3FB0020E9E710B50C000B8803700B8884
:106500001B0A43704B8883704B881B0AC3708A88B0
:106510000430063105F0B0FBA088043080B210BD15
:106520000420012B03D100201378009A13707047C8
:1065300010B50C000B8803700B881B0A43704A8847
:106540000230043105F098FB6088023080B210BD43
:10655000F0B589B003931E4B029242000700D05A57
:10656000019102F020F81325061E2DD0029B012474
:106570000370019B002B04D0001903999847001960
:1065800084B26B461B7A5BB2002B0FDA1021380005
:1065900002F01CFB1925002813D130003219E1B29A
:1065A00002F066FC051E0CD10C34A4B2042304AA2C
:1065B000380005A993800696948101F0AFFD051E71
:1065C00002D0300005F050FB280009B0F0BDC046F5
:1065D0005C67FF1F70B505000C0000280CD0002080
:1065E000814209D010222000044905F045FB01201A
:1065F0002B7823736B78637370BDC0466CC0001139
:10660000F0B506000D0017001C0085B002291BD054
:106610000020102907D1022B07D0102B03D115E041
:106620000020102C08D005B0F0BD69463800FFF7F7
:10663000D1FF2A0069460BE069463000FFF7CAFF28
:1066400022006946380004E0022BE9D12A00390013
:10665000300005F011FAE6E7031CF72800D9F7230C
:10666000032008499AB2013A0B80D3170340064928
:106670009B189B100B80D30F04499B185B100B8059
:106680007047C046A845FF1FA645FF1FA445FF1F32
:10669000034B1B888B4202D3024B4000C152704710
:1066A000A845FF1F5C67FF1F014B4000185A704749
:1066B0005C67FF1F1722014B1A8070475C67FF1F42
:1066C00070B505000E2005F0DFF8041E13D0D023AE
:1066D000037000230622837007494570033005F0DC
:1066E000CBFA064B2100DA8A62811B7E2373044BAE
:1066F000187805F079FA70BD7867FF1F6867FF1F8B
:10670000F845FF1F262803D8024B4000C05A7047A7
:106710000148FCE7AA45FF1FFFFF000070B5060017
:106720000C00094D1C220021280005F095F9074BAB
:106730001E70074B1C7005F0B7F90123002801D02B
:10674000002312202B7070BD6867FF1FF845FF1FE4
:106750008967FF1F70B505000D4C0800E260A1605D
:1067600010220021656005F0B7F9012803D110213E
:10677000A06802F058FD10220021280005F0ACF9B5
:10678000012803D11021606802F04DFD70BDC046A4
:106790006867FF1F70B5041E05D1002903D00622CB
:1067A0000D4805F069FA0D4B1D78012D11D1002C13
:1067B00005D102221A7005F0FFF9280070BD0022F1
:1067C0001A70074B1B78FF2BF7D02000FFF778FFDC
:1067D000F3E70025F1E7C0467867FF1F6867FF1FF2
:1067E000F845FF1F030010B5002801D1002010BD9F
:1067F00000780B4A002803D15988D1821B7913767F
:106800001378022BF2D10023984200D10333137086
:10681000044B1B78FF2B01D0FFF752FF0120E6E766
:106820006867FF1FF845FF1F002911D000280CD012
:106830004B79012803D140225242134303E03F2207
:106840001340032802D001204B7170474022F4E727
:106850000800FAE770B5094D0100287800280BD030
:10686000074C0622200005F007FA21002878FFF7E0
:10687000DBFF200005F0C0F970BDC0468867FF1F30
:106880006267FF1F00290AD0012808D13F224B79F7
:106890009343C02B03D0403B5A425341981C70474E
:1068A00070B5174D06002B78FF2B15D00A2004F089
:1068B000EBFF041E10D0D0230370C83B8370114B34
:1068C00011491B784670C3700622043005F0D4F9D4
:1068D0002100287805F088F90C4B1B78012B0DD18D
:1068E0000B4B1B68002B03D09B68002B00D09847F4
:1068F000084B04211878084A05F066F970BDC046B7
:10690000F845FF1F8867FF1F6267FF1F8467FF1F2F
:10691000B067FF1FB467FF1F60EA0000014B986873
:106920007047C0466867FF1F014BDB6818687047F7
:106930006867FF1F074B10B5DA68136801331360EF
:10694000054B1878FF2803D08021C90105F064FAAF
:1069500010BDC0466867FF1FF845FF1FF7B50E0062
:1069600002F0C8F8051E1CD00E4B06621F78002FDF
:1069700000D10778AB791020019304F085FF041E45
:106980000FD0D0230380C73B8370019BE91DC370E8
:106990000622043005F070F921003800E66005F0A9
:1069A00023F9F7BDF645FF1F014B18787047C04625
:1069B0008867FF1F054B002805D1054B1A78054B4A
:1069C000002A00D1014B18007047C0467867FF1FAE
:1069D0008867FF1F6267FF1F014B58687047C046FA
:1069E0006867FF1F024B1868431E9841C0B270478A
:1069F0008C67FF1F421E03000120152A03D9FF3BAD
:106A00005A425341D8B27047F0B51C0000230E0023
:106A100085B0039002920B70029A934201D300203A
:106A200019E0E55C5A1CD2B2002DF8D00298511939
:106A30008142F4DC0233DFB2A35C18000193FFF75C
:106A4000D9FF002807D0013D019A0399EBB23370BA
:106A50008A4202D1E01905B0F0BDDB19DBB2DBE7F9
:106A600010B50C0002F09EF803001220002B03D09A
:106A70002100588804F040FF10BD000070B50E4D95
:106A800084006359002B15D0186A002801D004F047
:106A9000EBFE2B59586A002801D004F0E5FE2B5973
:106AA000986A002801D004F0DFFE285904F0DCFECB
:106AB00000232B5170BDC0469867FF1F1C4B70B55B
:106AC00004000E00150099420AD11A4B1B68002BD6
:106AD00001D1122070BD1B68002BFAD09847F9E74E
:106AE000154B994215D1134B1B68002B0AD01B681C
:106AF000002B07D09847002804D1104B1C70104B76
:106B00001D70E7E729002000FFF7AAFF0028E1D168
:106B1000F3E7080001F0EEFF0028DAD00378032045
:106B2000A342D7D12900300004F0E6FED2E7C046E8
:106B3000FEFF00009467FF1FFFFF00009167FF1F2B
:106B40009067FF1FF7B50400808801F0D3FF002590
:106B5000A84203D00578A08802F008F81C4E3378CC
:106B6000002B1FD0AB421DD11A4B28001978FFF71C
:106B700077FF002818D000233370A3790820A77866
:106B8000A688019304F080FE011E0DD0D02303706F
:106B9000CA3B8370019B477086808371280005F093
:106BA00023F801E0002DE8D1A0880B4B8200D358D8
:106BB000002B01D0FFF762FF1721A088FFF768FDC7
:106BC000A08801F027FDA08801F0FEFDF7BDC046BA
:106BD0009167FF1F9067FF1F9867FF1FF0B587B091
:106BE0001D000CAB1B88070001930DAB1B88142004
:106BF00002930EAB1B88160003930FAB1B8800910A
:106C0000049310AB1B88059304F03EFE041E1AD0BB
:106C1000D0230370CB3B47708370C67006222900D7
:106C20000430002D11D005F027F8019B210063816D
:106C3000029B0098A381039BE381049B2382059B15
:106C4000A37404F0D1FF07B0F0BD04F005FFECE73A
:106C5000F7B5009308AB1B8807000C200D00160049
:106C6000019304F011FE041E13D0280001F042FF2E
:106C700000280FD00078D0232370C93BA370009B5D
:106C800021002381019B6770A580E680638104F069
:106C9000ABFFF7BD014B1878EDE7C046F845FF1F85
:106CA00013B5040064890389C2888188C078009480
:106CB000FFF7CEFF13BD000010B5044C206800287C
:106CC00003D004F0D1FD0023236010BD9C67FF1F9B
:106CD000A122F0B5818892004A43384B384F1B6897
:106CE00004009B189D2292009B18827989B01A603B
:106CF0003B68002B5FD01D78324B1B68002B04D003
:106D00005B68002B01D00020984726000836310030
:106D1000E079FFF7B7FD237DE0710200E07804938E
:106D2000638A29000393238A0293E3890193A3884A
:106D300000933300FFF752FFE378002B0BD1E28979
:106D4000A379A18802920196E2792800009201229B
:106D500001F0DAFEE0703B68002B20D0FFF7ACFFBB
:106D6000194D287800281AD0184B1978FFF778FEAB
:106D7000002814D02B78E67808200793A78804F021
:106D800083FD011E09D0D0230370CA3B4670837077
:106D900087808671079804F027FF00232B70172146
:106DA000A088FFF775FCA08801F034FCA08801F0F2
:106DB0000BFD09B0F0BD064B9DE7C0463409FF1F2F
:106DC0009C67FF1FB067FF1F9167FF1F9067FF1F42
:106DD000F845FF1FF8B5070008000E0001F08AFE15
:106DE000041E18D02620FFF78DFC051E00D1257843
:106DF000062004F049FD041E0DD00021062204F0F7
:106E00002BFED0232370C23B21006770A370A680A5
:106E1000E8B204F0E9FEF8BDF0B585B001930AAB25
:106E20001B78070002930BAB1B7808000D00009243
:106E3000039301F05FFE061E22D0102004F024FD13
:106E4000041E1DD01022002104F006FE2620FFF7AC
:106E500059FC002800D13078D0232370C13BA370A7
:106E6000009B21002372019B67706372029BA580C7
:106E7000A372039BC0B2E3720C9BE36004F0B4FE08
:106E800005B0F0BDF7B50D00019001F033FE071E0F
:106E900020D00E2004F0F8FC041E1BD02620FFF7A3
:106EA00031FC061E00D13E78D0232380C53B06224C
:106EB000A370F91DE01C04F0DFFE019B2A00638132
:106EC0000123DD401A401D40210022736573F0B29A
:106ED00004F08AFEF7BD0000F0B585B00290100006
:106EE0000D0017000A9E039301F004FE041E31D02A
:106EF000029B002B2ED1039B02795B0724D5122322
:106F000013430422002E08D10B99002905D10C99B6
:106F1000002902D10D9900291AD01A430D9B227124
:106F2000002B00D0C9E0002E00D1CFE0002D00D012
:106F3000CCE0606A002801D004F096FC1C213000EF
:106F400004F00AFD606205E002239A430E33D7E79E
:106F500093432371654BBA00D458002C00D1AAE0AA
:106F6000002E10D0236A002B03D11C2004F0ACFDAE
:106F700020625E4BBA00D358186A002803D01C2246
:106F8000310004F079FE0C9B002B12D0574CBB0053
:106F90001D596B6A002B03D1162004F095FD686221
:106FA000BB00E358586A002803D016220C9904F05D
:106FB00063FE0D9B002B11D04C4DBC006659B36A8B
:106FC000002B03D1142004F07FFDB0622B59986A86
:106FD000002803D014220D9904F04EFE380001F071
:106FE00089FD051E67D0414BBA00D358002B62D0F3
:106FF0001A6A3420002A00D11C389A6A002A01D06B
:10700000143080B20B9A002A01D01C3080B25B6A27
:10701000002B01D0163080B204F036FC041E4AD09A
:107020001822002104F018FD2620FFF76BFB0190C9
:10703000002801D12B780193D0232370029B2000DC
:1070400063700A23294EA370039BBD00A371AB5943
:10705000A780196A1830002905D01C22A06004F00E
:107060000BFE200034307359996A002907D00300C1
:1070700014221433E060029304F0FEFD02980B9B8F
:10708000002B08D003001C221C330B9920610293B3
:1070900004F0F2FD02987359596A002903D01622B0
:1070A000606104F0E9FD6B462100187904F09CFD55
:1070B0003800FFF7E3FC05B0F0BD10220D9B0D99E1
:1070C0001B69A018236204F0D7FD2CE70B9B002B53
:1070D00000D13FE7012D00D03CE7606A002801D0D5
:1070E00004F0C2FB1C210B982AE7C0469867FF1FDB
:1070F00010B5044C2068002803D004F0B5FB002331
:10710000236010BD8C67FF1F0B4B07B51A68002A60
:1071100001D100200EBD6946531C012012780731B1
:10712000FFF772FC0028F4D0027801231000184009
:107130001A42EED0EEE7C046A867FF1FF0B51F4F1A
:1071400001203B6887B0002B25D09B78059300F089
:10715000B3FB002821D00A20FFF7D4FA04000B204B
:10716000FFF7D0FA164B05001E78731E9E413B6850
:10717000F6B2191DD878FFF757FB3B682900DA7A79
:10718000043303929A790193029200903300200015
:10719000059A04F011FC07B0F0BDFFF7B5FF002819
:1071A00005D00620FFF7AEFA04000720D8E7082034
:1071B000FFF7A8FA04000920D2E7C0468C67FF1F3A
:1071C0008867FF1F70B50A4E040033780D00FF2B4F
:1071D0000DD0042004F058FB011E08D0D02303700A
:1071E000CE3B45708370C470307804F0FDFC70BDF8
:1071F0000846FF1F70B5040006200D0004F044FB94
:10720000011E0AD0D0230370CD3B8370054B447020
:107210001B688580187804F0E7FC002C01D0FFF78C
:1072200067FF70BD8C67FF1FF8B5264F06003B68EF
:107230000D001124002B05D10522234B1B7813428E
:1072400002D112242000F8BD204A10241268002A1E
:10725000F8D01278002AF5D0DB0719D52B789A1EC2
:10726000012A1AD80C2004F02FFC132438600028BF
:10727000E8D000230A22437029000670023004F08F
:10728000FBFCFFF75BFF041E0AD0FFF731FFD9E7D5
:1072900000F012FB0028E1D1E4E7002BE2D0D0E7B8
:1072A0000B4B1B78032BCDD11D20FFF72BFA094B7D
:1072B00018800028C6D0084B04211878074A04F02B
:1072C00083FCBFE78C67FF1F8967FF1FA867FF1F4D
:1072D0008867FF1F8667FF1FB467FF1F60EA000013
:1072E000F7B50193194B14001A78052306000F0017
:1072F00012201A4221D0012920D1154B1D68002DE2
:107300001BD002201F2C18D8002C02D0019B002B70
:1073100013D0104B1F221E706E1C0021300004F091
:107320009BFB01992200300004F0A6FC31002000F4
:107330002C70002F06D004F04FFDFEBD064B12202E
:107340001D68DCE704F0E8FCF7E7C0468967FF1F2B
:10735000A867FF1F0846FF1FA467FF1FF8B50F4E61
:1073600012243368002B17D01B780F3C834213D1B3
:1073700000250B4F0221387804F0E6FA094B04216E
:1073800038781D8004F0E0FA074B28001D80336830
:107390005C7004F0F9FA04002000F8BD8C67FF1F50
:1073A000B467FF1FA067FF1F8667FF1F70B5012826
:1073B00023D11B4C2388002B03D01A4A1578002DAB
:1073C00007D0194B1B68002B02D01878FFF7C6FFB7
:1073D00070BD3B2B02D93C3B2380F9E7134E0221C1
:1073E000307804F0B1FAFA222388920002215A433D
:1073F000307804F031FA2580EAE70B4B1B68002B4C
:10740000E6D00B4B1B785B07E2D5084B02211878BE
:1074100004F09AFA0022024B1A80FFF769FED7E7C0
:10742000A067FF1F8467FF1F8C67FF1FB467FF1FE4
:107430008967FF1FF8B51E4D2868002803D004F0A7
:1074400013FA00232B601B4E3068002803D004F091
:107450000BFA00233360184F05243B7818002040B6
:10746000234221D0154800F02BFA3B78234213D059
:10747000202004F029FB2860002813D020220021BE
:1074800004F0EAFA202004F01FFB041E306005D04F
:107490002022002104F0E0FA002004E0286804F033
:1074A000E3F92C601320F8BD00F00AFAF4E7C046B7
:1074B000A867FF1FA467FF1F8967FF1FFC45FF1F09
:1074C00010B50A4C23681A1E0ED0002808D10130CE
:1074D000587004F059FA002805D02368002B02D018
:1074E0000021FFF787FE0122100010BD8C67FF1FEF
:1074F000F7B5274E050033680191181E21D05C783E
:10750000244F012C30D1FFF7FFFD002825D02000AB
:10751000FFF7F8F80400412814D91F4B022118780E
:107520001E4A04F051FB1E4B3C3C1C800222336877
:107530005A703B78002B14D128000199FFF75AFEAE
:107540000120FEBDFA2292004243002AEED0124BE7
:107550000221187804F080F9E8E7FFF7D3F8020079
:10756000F3E700233B70EBE73B78002BE8D10320E7
:1075700004F08AF9011E08D0D0230370CC3B45707B
:1075800083703368187804F02FFBFFF7B1FDD7E75D
:107590008C67FF1F8467FF1FB467FF1F60EA00004E
:1075A000A067FF1F10B51749838802008B4220D0C7
:1075B00011D815498B4217D0144900205B1899B295
:1075C000012907D8926811785A425341D8B2FFF77F
:1075D000F9FD012010BD0E4A00209B1807229BB226
:1075E0009A424041C0B2F5E783681878FFF768FF18
:1075F000F0E7836899785A78090218781143FFF701
:1076000077FFE7E70A20000006200000F8DFFFFF11
:10761000AFDFFFFF014B18707047C0460946FF1FE0
:1076200010B5064C207001F041FA207804F03CF9C6
:107630000521207800F062FD10BDC046B467FF1F31
:107640000BB273B50D00002B00DBC4E0884B18783B
:1076500004F05AF9041E0ED00378912B0FD0A22B00
:1076600000D1A1E0834B1878FF2852D0210004F00C
:10767000BBFA00284DD180200002684076BD4378D7
:107680000F2B76D013D8052B70D00E2BEAD1808823
:10769000794B98422BD8794B98421BD8784B98421B
:1076A000E0D1A3681878591CFFF774F838E03E2B36
:1076B000D8D18378032B74D06CD8012B6ED0022BD9
:1076C000D0D1704B1B68002B23D05B68002B20D0DF
:1076D00098471EE06C4BC0180C28C3D804F04CFB34
:1076E0001DC2C2150BC20B0B0B3223C23C00674BF1
:1076F000C0180728B6D8664B1B68002B09D01B683A
:10770000002B06D0200098470AE0A3681878FFF7FE
:10771000C7F8200004F0E8F9ADE7A068FFF762F8C9
:1077200000289FD0F5E7A3681B78002BF1D0554BBC
:107730001B68002BEDD01B68002BEAD021005548B8
:107740009847EDE74F4B1B68002BE2D01B68002BDE
:10775000DFD021005048F3E7504B1B68002BD8D0F6
:107760005B68002BD5D021004348E9E7FFF7EAF931
:10777000CFE780884A4B984203D04A4B984200D0CA
:1077800070E7464B1B68002BC3D05B68002BC0D052
:107790002100D5E7153B012BBBD963E7FFF798FA2A
:1077A000B7E7FFF77DFAB4E73F4B1B78042B07D10F
:1077B00000236A4613800179408800F0C5FCA8E7E1
:1077C000364B1B68002BA4D05B68002BA1D00100B6
:1077D000364898479DE7012421420AD0294B1B686F
:1077E000002B04D05B68002B01D0002098470120BB
:1077F00043E78B070AD5264B1B68002B04D05B6838
:10780000002B01D020009847022036E704212800F1
:1078100008400D4200D131E7254E3388002B21D09E
:10782000013B9BB23380002B1AD1FFF7DBF8002815
:107830000AD0204B1C70164B1B68002B04D05B68D1
:10784000002B01D020009847FFF7C6F8694601F0E9
:1078500001FD6846FEF7FEFF1D20FEF753FF308056
:1078600004200AE7024B187804F06EF8F8E7C046E7
:10787000B467FF1F0946FF1F0E2000000120000013
:1078800009100000AC67FF1FFEDFFFFFAFDFFFFF47
:10789000B067FF1F0C2000000B2000009467FF1F43
:1078A0000D200000132000008967FF1FFFFF00006C
:1078B0008667FF1F8467FF1F10B501F09BF910BD9D
:1078C000014B18607047C046B067FF1F0B8800204F
:1078D000162B01D817230420014A13807047C04695
:1078E0005E67FF1F00207047074A0300118881422E
:1078F00007D091880020994202D1013080001018F1
:1079000070470020FAE7C046BC67FF1FF0B58F78CC
:1079100006000D00C7B01E2F15D1FFF7E5FF051EAD
:1079200003D10024200047B0F0BD00223B0031000D
:10793000C078009200F0B2FB0400A81C00F0D3FB5A
:10794000FF23EB70EEE7264B062403931B78FF2BF7
:10795000E8D0182FE6D87B08224A013BDB000292D0
:107960009A589446002ADDD0029AD3185B68002BFF
:10797000D8D00878002802D14B78012B02D10624F8
:10798000122FCFD107AFAB88697800976446AA68F9
:10799000A047041EC6D1AB78029A5B08013BDB000E
:1079A000D318390030005B689847041E0BD1AB78C0
:1079B000042BB6D0039A310010782200009700F013
:1079C0006DFB0400AEE76A78002AABD1AA7805A95E
:1079D0003B88087130000A704B80FEF747FBA0E738
:1079E0000C46FF1F7CC000111D4B37B505009842A7
:1079F0000BD000290AD1FFF777FF002805D11948DD
:107A0000FFF772FF002800D0058037BD01291AD189
:107A1000FFF76AFF041EF8D001235B420380A378BE
:107A2000FF2BF2D0FE2B07D00023E0781422009326
:107A300029001E3300F032FBA01C00F054FB012390
:107A40005B426380E1E70229DFD1013901F0BEF832
:107A50000028DAD12800FFF747FF041EDFD1D4E762
:107A6000FEFF0000FFFF0000022210B5074B52424C
:107A70001A80074801325A809A80DA8000F07EFA34
:107A8000044801F025F8002010BDC046BC67FF1F68
:107A90000D790011E97900110388F7B50400002B76
:107AA00002D102252800FEBD426802211378254834
:107AB0005268FEF7A5FD00282ED0234F01253A88F5
:107AC000002AEFD0802321885B0201259B1A99426E
:107AD000E8DC0C2003F0F8FF061E31D03B8822883A
:107AE0009C4600231800019561469DB2491989B250
:107AF000AA421BD8002801D062443A8000233000FB
:107B0000082208C0210004F0B7F8104A1368002BBF
:107B100013D100251660C5E76268022113780C486E
:107B20005268FEF76DFD0028C7D1BAE760681D01F5
:107B30004019418101330198D6E71A001B68E6E736
:107B40001325AFE7EAC000110A46FF1FB867FF1F01
:107B5000E8C00011014B18707047C0460C46FF1F6B
:107B600014230A0010B51A40194204D00122102132
:107B700001F048F810BD4B06F9D4012088434000BD
:107B8000F8E710B514008B0604D50122102101F08E
:107B900039F810BD08230A001A40194202D14BB22D
:107BA000002B0FDA102101F02DF8002808D0230057
:107BB000F9331B78002BECD0F8342378012BE8D173
:107BC0000020E6E703208907FAD4E2E7F0B51F00BA
:107BD000184B85B01C68019002910392002C27D1AC
:107BE000200005B0F0BDA5683301ED186B89019A3E
:107BF000934211D3029A93420ED8002F04D10A9BCC
:107C0000002B10D12C00EBE73B002978039A686821
:107C1000FEF7F6FC0028F2D10136B6B2A388B342D3
:107C2000E1D82468DAE7A3680A9A5B891380E9E758
:107C30000026F3E7B867FF1F37B50C000A884988AC
:107C40000123914217D3002A15D0651D23792A00FC
:107C500002210A48FEF7D4FC102300280BD0237918
:107C60006188208800242A000094FFF7AFFF0A23D0
:107C7000A04200D0230018003EBDC046EAC000115B
:107C800013B50A0008884988012388420BD80028C8
:107C900009D00024137905320094FFF797FF0A23D7
:107CA000A04200D02300180016BD13B50A000888B2
:107CB0004988012388420BD8002809D00024137971
:107CC00005320094FFF782FF0A23A04200D0230070
:107CD000180016BDF0B58BB003904A8808880E00D6
:107CE0000123824255D3002853D00023012704AC3E
:107CF00023700022718813000092FFF767FF051EB2
:107D00003ED02078002835D12B78022B18D167700F
:107D10006A8983000130E31880005A806968022272
:107D2000201803F0A9FF23780133DBB22370042B62
:107D300019D93B006889013080B2002BD9D01FE0EF
:107D400002236370122358436A89231804305A802F
:107D500069681022201803F08FFF23780133DBB20B
:107D60002370002BE5D10C4A6B899B185A42534172
:107D7000DBB2DFE76378012BE4D12B78022BC7D08D
:107D800022780A23002A04D021000398FEF798F9EC
:107D9000002318000BB0F0BD0100FFFF0F4BF0B542
:107DA00004001868002816D083685D89A54207D8AA
:107DB0008288AE18B44203DA12019A18934201D1B4
:107DC0000068EFE71E005F891036A74204D1002942
:107DD00000D00D801800F0BD3300EFE7B867FF1F3B
:107DE00070B505000C0008880021FFF7D7FF0300DD
:107DF0000120002B04D022002800197AFFF7C1FED1
:107E000070BDF7B50C00002501902300F6331B78F8
:107E1000AB4201D800200AE06B00E65A0021300096
:107E2000E718FFF7BBFF002802D126800130FEBD16
:107E3000017A0198FFF794FE002802D03B88238046
:107E4000F5E70135EDB2E0E710B504000888002140
:107E5000FFF7A4FF03000120002B03D02000197AB4
:107E6000FFF77EFE10BD0000054B1B68002B01D103
:107E7000180004E09A6852898242F6D198887047C7
:107E8000B867FF1FF0B50E27002687B0039302AB3B
:107E9000FF183E8005001F4B40891400984207D010
:107EA0002B78013000976A6880B2FFF78FFE0600DA
:107EB00002212B7818486A68FEF7A2FB00280FD031
:107EC0006C892000FFF7D0FF002802D0013C041984
:107ED000A4B2039B002B00D01C80300007B0F0BD83
:107EE00002212B780D486A68FEF78AFB0028E7D14B
:107EF00002212B780A486A68FEF782FB002807D027
:107F0000002EDED03B88A342DBD17489013CDFE741
:107F10006C89DEE7FFFF0000EAC00011E8C0001135
:107F2000E6C0001110B50C00FFF7DEFC03000220D4
:107F3000002B0AD0002C00D023609B781720FE2B4A
:107F400003D00138FF2B00D1002010BD73B50D0008
:107F500001A904001600FFF7E5FF172805D0002E41
:107F600004D129002000FEF727F976BD0122102157
:107F7000200000F047FE0028F3D0F6E7014B186020
:107F80007047C046C867FF1F37B56B469D1D01008F
:107F900004000222280003F0CFFD2B88B02B0ED165
:107FA0002379122B09D12300FF339B78012B06D1B3
:107FB0000121608800F0E0F801E01B2BF8D037BD0C
:107FC00010B5054B0421187000F098F8FFF74CFD30
:107FD000FEF770FB10BDC046CC67FF1F0020F0B558
:107FE0000BB20F0087B0834234DA274B187803F0C6
:107FF0008BFC051E2BD00378A02B25D103AE3100BE
:10800000FEF7E4F8041E0BD1B378DB0724D51F4B31
:1080100006341B68002B03D03100688898470400A1
:10802000A868002801D003F01FFE002C08D1184AD0
:10803000039B1340174A934206D0B3781B2B03D0FF
:108040000121688800F098F8280003F04DFD802099
:108050000002784007B0F0BD0F4B1B68002B10D01A
:10806000310068889847041EDAD07378002BD7D186
:10807000B27801A90A704B800C716888FDF7F6FF91
:10808000CEE70624F1E7C046CC67FF1FC467FF1F99
:1080900000FFFF0000011200C867FF1FF7B5019045
:1080A000822040000D0017001E0003F0EDFB0400CD
:1080B0001320002C12D0B02320002370089BFC2238
:1080C0006770658026710830002B08D0190003F016
:1080D000D3FD2100019803F087FD0020FEBD089923
:1080E00003F0BAFCF5E710B5041E06D00078FD28B1
:1080F00003D803F0E9FDFF23237010BD0A1F93B2DC
:1081000010B504000220032B05D882400020024B4A
:10811000D1529B189C7010BDEC67FF1F0B8870B587
:10812000043B04000D000220032B0BD8012120008A
:1081300000F04CFD03001420002B03D02900200088
:1081400000F0DEFB70BD000007B51300034A00928B
:108150000A00012100F02CFC0EBDC04685830011F1
:1081600007B5019203220092024B0A00122100F08F
:1081700049FC0EBD0384001107B56B4601AA1180AE
:108180000449D88008780633012802D1190003F089
:108190000BFC07BDCD67FF1F0C4B10B518700023FB
:1081A000FF210B4A1380138193819380094A5380E6
:1081B0001370517293819372D174D3821375517776
:1081C00003F0EAFC00F0FCF910BDC046FC67FF1F9D
:1081D000EC67FF1FCE67FF1FF0B58DB06B46002028
:1081E00003910C229B5E834200DBB0E05D4B18786C
:1081F00003F08AFB051E00D1A4E00378902B00D089
:108200009DE006AF01004688380000F013FA796857
:108210000400002900D19CE03B88052B6ED13B89EE
:10822000032B1CD905AC200000F0A2F86288172AA5
:1082300061D83989131D994231D179682378043185
:108240000291D90738D5607800F08EF9071E06D064
:10825000002303712378012B08D0132B23D0A868A7
:10826000002800D178E003F0FFFC75E062880299F5
:1082700009A800F0A6F80290380000F08BF909AACE
:108280002378387A0192002231000092029A00F09D
:1082900012F9380000F064F9029B002BDFD03000A7
:1082A00000F080F9DBE70378032BD8D162880299CC
:1082B00009A800F0D6F8DEE7122B13D1029909A81D
:1082C00000F0B5F8021EEAD127498B88002BC6D0F2
:1082D000887909A92378019161780091310000F033
:1082E000EAF8BCE7002302AA93833000617809AA68
:1082F000FFF72AFFB3E71D4B0993F6E7042B02D0E3
:108300009A1F012AABD8184A043B9B00995A0029AE
:10831000A5D0D218907831003A0000F0AEF80028CD
:108320009DD13B88042B03D001213000FFF724FFAF
:10833000012C04D1A868002801D003F095FC280086
:1083400003F0D2FB8020039B0002434018000DB0D5
:10835000F0BD012800D182E701213000FFF70CFFBA
:10836000EDE7C046FC67FF1FEC67FF1F0100170029
:108370000B7803704B784370CB788A781B021343D9
:10838000438070470A88030002700A88120A42700C
:108390000A88012A06D14A8882704A88120AC27065
:1083A0000420704702208242FBD14A8804309A7030
:1083B0004A88120ADA708A881A718A88120A5A71EF
:1083C000EFE710B50400012082420CD94B780A78FF
:1083D0001B0213432380834206D1CB788A781B0289
:1083E00013436380002010BD022BFBD1CB788A7829
:1083F0001B02134363804B790A791B021343A3804A
:10840000F0E70B8803700B881B0A43704B8883705E
:108410004B881B0AC3708B8803718B881B0A4371BE
:10842000CB888371CB881B0AC37108207047030077
:108430000120082A14D14A780878120202431A80CF
:10844000CA788878120202435A804A79087912025F
:1084500002439A80CA798879120202430020DA80A6
:10846000704710B504000120022A05D100204B7886
:108470000A781B021343238010BDF8B506001020B4
:108480000F00150003F000FA04000120002C0ED0AC
:10849000A0230C22290023806780201D002D07D0F7
:1084A00003F0EAFB2100300003F09EFB0020F8BD42
:1084B00003F0D2FAF6E7F7B51E00009008AB1420DF
:1084C00017001D78019103F0DFF9041E12D0A223DA
:1084D0000370019B47704380099B057146710C2214
:1084E0000830002B07D0190003F0C6FB21000098CC
:1084F00003F07AFBF7BD099903F0AEFAF6E737B55A
:10850000041E0FD04388002B0CD00025C1881323F4
:10851000007A172201950095FFF7CDFFFF236580B4
:108520006372257037BD000010B50C4904004A88FD
:10853000002A09D08B89002B05D00020CB8A02228B
:10854000834201D010BD012213000A2043430020C2
:108550004032C854C81842800472F3E7CE67FF1F48
:108560000023438003707047094B00211A0010B5A7
:108570005C88002C06D01C79844203D10A234B432B
:10858000D01810BD01310A330329F1D10020F8E7DA
:10859000CE67FF1F10B50400407A03F095FBFF2360
:1085A000637210BD7047043010B580B203F03CFB1D
:1085B000002803D00421494203F066FA10BD0000F0
:1085C00070B50025104CA0682580A581A580A84223
:1085D00002D003F049FBA56000250C4C0C4B606DEC
:1085E0001D80230058331D70A84202D003F03CFBCD
:1085F000656500256068002801D003F035FB013572
:1086000008340A2DF6D170BD9468FF1F3868FF1F2B
:108610008868FF1F70B5041E09D1054D2880A88108
:10862000A880A868002802D003F01EFBAC6070BDD3
:108630009468FF1FF0B54B8885B001930023436019
:108640000A7905000F00022A00D07BE0CA88032ABD
:1086500017D98B685E7819783602DC78D8790E43A2
:1086600099781B7A24021B020C43034353495BBADB
:108670000B80331D93421ED1042C04D0631F022BA8
:108680000ED9012015E0019A4D4B1201D35A002B4F
:1086900006D00198FFF7BEFF4A4A13690133136100
:1086A0000421B8682E812C80494203F0EDF96860FE
:1086B000002005B0F0BD434D042C06D0631F022BF3
:1086C0000FD9EB680133EB60DBE7019A3C4B1201F9
:1086D000D35A002B05D00198FFF79CFF2B6901337B
:1086E0002B61374B30000293019B029A1B010193CF
:1086F000002301998C468B52130063449C800393A2
:108700009E81FFF750FF039B041E986016D0042142
:10871000B868494203F0B8F9FA880100043A200029
:1087200003F0AAFA0199029AFB888A5A043B9B1823
:10873000029A8B522B6801332B60A2E7AB6901339D
:10874000AB619EE71E4B0293019B1E01029BF35AF5
:10875000002B2DD002998C19A068002828D0012A5E
:1087600026D1FA889B189BB27352A189994217D3DC
:108770009B1AC018B96803F07FFA029BA289F35ACA
:10878000934200D07DE700222B81A3882B80A36831
:108790006B60029BF2520B4A53680133536070E7DF
:1087A000084A9368013393600198FFF733FF68E745
:1087B000044A536901335361F6E7C046FE67FF1F61
:1087C0009468FF1F0468FF1F70B5051E15D10B4C80
:1087D0000B4B1880230058331870606D002802D0AE
:1087E00003F042FA6565250050356068002801D025
:1087F00003F03AFA0834AC42F7D170BD3868FF1F75
:108800008868FF1FF0B51700A12285B09200019380
:108810004243394B06001B680C009B18D933FF33C9
:108820001D78FDF741FF0430854204DD3000FDF77F
:108830003BFF0430C5B2BD4207D33A0000213000EF
:10884000019B02F0D1FF05B0F0BD2900380003F014
:10885000A3F82300C6B250331E700393019B290076
:108860006365380003F0A0FACBB20293002B02D06C
:10887000039B01361E7000262300503303931B78A0
:10888000B34204D8606D002831D10020DBE7029AA2
:108890002800002A04D0013B1000B34200D0280079
:1088A000F700E719387003F04FFA786000280ED00F
:1088B0003A78019903F0E0F9019A3B780136D31830
:1088C0000E4A0193D369F6B20133D361D4E7039B17
:1088D00018706065A74205D1084A1320D36A013396
:1088E000D362B0E7606803F0BFF90834F2E703F041
:1088F000BBF900236365C8E73409FF1F0468FF1F45
:10890000F7B50D0007000421686803F0BDF82B8956
:10891000040003702B891B0A43702B8883702B88FB
:108920001B0AC3702E8902250436F6B2FB2E15D819
:108930001B4B9F4214D10C2002F0A6FF1135011EE3
:108940000CD0902303708E3B0371043B4380154B86
:108950008460C680187803F047F900252800FEBD22
:108960005C237B43104AD3180093583301931B7840
:10897000002B0FD10300320038000099FFF742FFAF
:10898000019B05001B78002BE8D13800009903F00B
:10899000A3F9E3E7054A0725536A01335362DDE78C
:1089A000FEFF0000FC67FF1F3868FF1F0468FF1F01
:1089B000F0B587B0009017200F0016000193FFF765
:1089C000F2FD1325041E19D00C98031E02D0019944
:1089D000201D9847030AE370052302AAA070043003
:1089E000908127700098667003A993800494FFF724
:1089F00087FF051E02D0200003F036F9280007B0DB
:108A0000F0BD0000F0B587B01F000CAB1B780391E0
:108A1000059301210DAB06001C78049200F0D6F8F6
:108A20001425002821D02000FFF77EFD0135041E0B
:108A30001BD01149059B0A7803700132D2B2131E74
:108A4000C68001D101231A000B7022713000049BF3
:108A500003990097FFF7ACFF051E09D12300210001
:108A60000648074A093302F0C7FF280007B0F0BDE7
:108A7000002363802370F8E70068FF1FFF84001164
:108A800030750000F8B505000E00064C064F23684F
:108A9000002B02D03100280098470434BC42F6D1A4
:108AA000F8BDC046A468FF1FB868FF1F0123064A2F
:108AB0005B425380002313715362044A1360536076
:108AC0009360D36013617047B868FF1FA468FF1FED
:108AD0000200002310B506499C000859002801D166
:108AE000625010BD0133052BF6D11320F9E7C046C3
:108AF000A468FF1F034A5388181A43425841404252
:108B000010407047B868FF1FF0B585B002930AABFC
:108B10001F780CAB1B88009008000E000192039395
:108B2000FFF7E8FF05001120002D1BD10E48FFF7CD
:108B3000E1FF04001520002C14D006220B99A77128
:108B4000E01D03F099F8019B30002371029B29007E
:108B50006371009B66802370039B6562E381FFF76E
:108B600091FF280005B0F0BDFFFF000010B5FFF732
:108B7000C1FF04000220002C12D060880121FFF701
:108B800081FF606A002801D002F06EFE28220021D9
:108B9000200002F061FF012300205B42638020710E
:108BA00010BD000030B5074A074C55880100137806
:108BB0000020A54204D05B1A59424B415842104054
:108BC00030BDC046B868FF1FFFFF0000084A10B55F
:108BD00001230C00904208D0FFF78CFF031E04D045
:108BE000037923405A1E9341DBB2180010BDC046E2
:108BF000FEFF0000024B1879431E9841C0B2704737
:108C0000B868FF1F70B504000D001600FFF772FF73
:108C1000002804D10D4B9C4200D0143070BD416A35
:108C200003790520002907D012221A40102A02D108
:108C30000520002EF2D10F20DB06EFD5897E0C2017
:108C4000A9428941494249420840E7E7FEFF000046
:108C5000030010B5002800D110BD0348034A418825
:108C60009142F9D09847F7E7B868FF1FFFFF00006F
:108C7000002330B5C45CCD5C6C40D4540133102B60
:108C8000F8D130BD0F23002210B5C45C640022432C
:108C9000CA54C25CD209013BF7D210BD02000100E8
:108CA00010B52032103102F0F7FF10BDF0B58BB0D7
:108CB0000390102005931700049102F005FF009027
:108CC000102002F001FF009B13240190002B05D01F
:108CD00000280CD11324009802F0C6FD019B002B44
:108CE00002D0180002F0C0FD20000BB0F0BD102033
:108CF00002F0EAFE0600102002F0E6FE1324050052
:108D0000002E00D1AEE0002819D01022002102F080
:108D1000A3FE32002900039802F0BEFF041E0ED10C
:108D200033787F2B51D830000099FFF7ABFF009BC1
:108D30001B787F2B53D801990098FFF7A3FF3000D1
:108D400002F092FD002D02D0280002F08DFD002CD3
:108D5000C1D1102002F0B8FE0600102002F0B4FECF
:108D60000290002E7CD0002878D03A000F322300E9
:108D70000125121105D00F333B4015B25A42534121
:108D80001BB26A1E1201002B33D0049BD2B298187A
:108D90000099029AFFF76CFF013D1022002130007C
:108DA00002F05AFEADB2049F2D017D19AF4242D0B0
:108DB000002C33D0300002F057FD029B002B00D175
:108DC00089E7180002F050FD85E729003000FFF721
:108DD00059FF28002549009AFFF74AFFA7E7290015
:108DE0000098FFF74FFF28002049019AFFF740FF46
:108DF000A5E70F210F4004998A18D9B28F4208D9EC
:108E0000D15C06A819540133102BF6D1029A0199AE
:108E1000C0E7791A48424141C901F2E73900300000
:108E200006AAFFF725FF3200039806A902F034FFD7
:108E300010370400BAE7002CBCD13000029906AA12
:108E4000FFF716FF320006A9039802F025FF08225B
:108E500004003100059802F00FFFABE71324A9E7E7
:108E60001324AAE7002800D06EE733E7F0C0001112
:108E7000F0B58BB00F0016000225009000283FD0FF
:108E8000002A3DD00B1DDBB21800029302F01CFE3D
:108E90001135041E34D0FDF747FD05003A00009956
:108EA000201D02F0B9FEEBB20393E3702B0CDBB292
:108EB0002F0A00936370FFB22B0E2370A7700193EB
:108EC000FDF72CFD1022010006A802F0A5FE2100EE
:108ED000029A04AB06A8FFF7E9FE051E0DD1039B1D
:108EE00008223370009B04A9B370019B7770F37064
:108EF000301D02F091FEFDF71DFD200002F0B4FCD4
:108F000028000BB0F0BDF0B58FB00D00149E03909B
:108F100004920593002A03D1022420000FB0F0BD73
:108F2000002EF9D00398FFF7E5FD1424071EF4D0B6
:108F30007278337812021A43B3781B041343F27821
:108F400012061A43036A0192934201D30133E3D11B
:108F5000002D03D03B7901249B07DED50822002198
:108F600006A802F079FD059B13240433DBB2180038
:108F7000029302F0A9FD051ECFD0059A0499043092
:108F800002F04AFE04223100280002F045FE3900BA
:108F9000102210310AA802F03FFE2900029A06AB07
:108FA0000AA8FFF783FE041E0FD1082206A908A80D
:108FB00002F032FE0822311D08A802F05DFD0128F2
:108FC00007D101990398FDF7C9FC280002F04CFC79
:108FD000A3E70124F9E7000070B51C4C05002368E5
:108FE000181E10D0002D14D11A78002A0CD1981C0C
:108FF000083202F041FE02F07FFE0135002808D160
:1090000023681D70012070BD0A331800082202F089
:1090100033FE2368002BF5D0122002F035FC061E2B
:109020000DD0C12321680370457002311022023037
:1090300002F022FE23683100587802F0D5FD206846
:1090400002F012FC00232360DCE7C046E068FF1F4B
:10905000F8B504002020FDF755FB0D4EA700BB59C5
:109060000500002B0DD000280BD0D878FF2809D19F
:1090700008492A000C55F35907480333611802F0D8
:10908000BBFCF8BD290002F0DFFC0028F0D1F8E7B6
:10909000FC68FF1FE468FF1FA9A2001170B5064D10
:1090A00084006359002B05D0D87802F00DFEFF2212
:1090B0006359DA7070BDC046FC68FF1F70B50600CA
:1090C0008CB00C00150000213022684602F0C4FC70
:1090D00031001022684602F09FFD1D20210003226E
:1090E000684402F099FD6846FFF7D8FD2D21040081
:1090F00003222800694402F08FFD20000CB070BDEF
:10910000F0B50700160097B001931CAB1D78302214
:109110001EAB00910AA800211C7802F09DFC1022D1
:1091200039000AA802F078FD1022002102A802F0FE
:1091300093FC0722310002A802F06EFD072202AB69
:109140009818631E9C41019902F066FD02AB9C7366
:109150002B005A1E934102AAD3730021102206A8A5
:1091600002F07AFC06221D9907A802F055FD1A208C
:1091700002ABC01806221F9902F04EFD1022009982
:109180000EA802F049FD102202AB0EA908781C7847
:10919000013A6040D2B2087001330131002AF5D1A2
:1091A0000AA8FFF77BFD102212A904000EA802F006
:1091B00063FD102206AB0EA908781D78013A6840BD
:1091C000D2B2087001330131002AF5D10AA8FFF7A5
:1091D00065FD044310222098E4B212A902F01CFDA0
:1091E000200017B0F0BD70B50E0014008CB0010067
:1091F000102268461D0002F00FFD3100082204A86D
:1092000002F00AFD2100082206A802F005FD6846CA
:10921000FFF744FD04001022280008A902F0FCFC1E
:1092200020000CB070BDF8B506000D000024371901
:10923000AC4200D3F8BD02F0FFFA030A3B70631C96
:10924000DBB201379D4203D90234F054E4B2EEE7B9
:109250001C00EDE773B506000C000225002819D0AC
:10926000002917D0032101A8FFF7DDFF6B469A798B
:109270003F231A40013313436A463000937101A91A
:109280002200FFF71BFF051E04D10322E01C01A9E9
:1092900002F0F2FC280076BD03785807DA08C00F08
:1092A000D20080009B0710439B0F1843C0B2704749
:1092B00007230B40C908C9000B4303707047000027
:1092C00070B50400FFF7EAFE134DA4006359002BAC
:1092D00021D0186A002801D002F0C6FA2B59986EE6
:1092E000002801D002F0C0FA2B59D86E002801D016
:1092F00002F0BAFA2B59186F002801D002F0B4FA24
:109300002B59586F002801D002F0AEFA285902F00C
:10931000ABFA00232B5170BDFC68FF1F0E4B800081
:10932000C35870B50C00002B0FD09D68002D0CD0D9
:109330002B78201D0B706B784B70A97CFFF7B8FF62
:109340002B7E23726B69E36070BD10220021200028
:1093500002F082FBF8E7C046FC68FF1F014B186073
:109360007047C046F868FF1F074A03008000825814
:1093700010B5002A06D0D088984203D1012901D126
:10938000FFF79EFF10BDC046FC68FF1FF0B5264EDC
:1093900095B087000B93BB590500099112200A92E2
:1093A000002B31D0D888FFF7A5FB04001420002C37
:1093B0002AD0280010A9FFF7B1FFBB591E781D6AFB
:1093C000002E23D00895FDF7EFFA07000020FDF7E7
:1093D000F1FA0790A379E61D069310AD0CA9089841
:1093E00000F0E2FA0EA9280000F0D7FA0B9B0A99C8
:1093F0000493069B09980293079B03960193009799
:109400000EAB0CAAFFF77CFE15B0F0BDFDF7CCFA51
:1094100006903000FDF7CEFAE31DA779079310AB55
:1094200006000893DAE7C046FC68FF1F30B50C4C15
:1094300085002A59030085B00120002A0ED01800AB
:109440006946FFF76BFF2B591A78D888054B002A1D
:1094500000D1054B6A46072100F0D9FB05B030BDAD
:10946000FC68FF1F9B990011A999001130B5094CA8
:109470008500295985B010226846253102F0FCFB91
:109480002A591121044BD0886A4600F0C0FB05B070
:1094900030BDC046FC68FF1F459A001130B5094C2D
:1094A0008500295985B010226846353102F0E4FB69
:1094B0002A591121044BD0886A4600F0A8FB05B058
:1094C00030BDC046FC68FF1F839A0011F7B54D4FB1
:1094D00086001020F4590D0002F0F6FAF3592062CC
:1094E000186A132200286CD0033A29009C6802F005
:1094F000C3FBF3591A780192002A58D11E6A227DC3
:10950000317B944651400122019F114201D16746AF
:109510001740217D914339432175377B4F40BC462D
:1095200060460027800701D44F0817400121022020
:109530008F40227D82433A432275377B5740BC4699
:1095400060460027400701D497080F400420227D81
:10955000BF0082433A432275627D002794466046ED
:10956000727B42400A4201D167460F400121627D71
:109570008A433A436275777B5740BC466046002772
:10958000800701D457080F400220627D7F0082438C
:1095900017436775767B00227E40760701D4BA08B0
:1095A0000A400426617D9200B1430A4362756A78DD
:1095B000002A08D06278002A05D005220533DA7720
:1095C00000221000FEBD04222979114205D1A17CA0
:1095D000114202D10533033AF1E7019A21782C7840
:1095E000002A02D10A002100140018220429E8D818
:1095F000042CE6D805206043034A05331218525C58
:10960000DDE7C046FC68FF1F00C1001110B50A006D
:109610001121024B00F0FBFA10BDC046DF9A001189
:109620000B0030B587B001AD2B806B4604001100F4
:10963000981D082202F020FB2A000B212000024B7B
:1096400000F0E5FA07B030BD079B001110B50A0025
:109650001121024B00F0DBFA10BDC0465B9B0011EC
:1096600013B50B0011006A4613706B460400062206
:10967000581C02F001FB6A4608212000014B00F053
:10968000C6FA13BD7B9B001110B50A001121024BD5
:1096900000F0BDFA10BDC046CB9B00117FB50500A0
:1096A0000B4BAA00D4580800002C0FD0666F237F04
:1096B000E28821780396266F0296E66E0196A46EE4
:1096C0000094FDF709FC2800FFF7FAFD7FBDC046B6
:1096D000FC68FF1F10B51721FFF7E0FF10BD000069
:1096E00070B50A000D00064B0221040000F08FFA4D
:1096F000060029782000FFF7D1FF300070BDC0467A
:10970000AB9A001170B586B000236A461370836867
:1097100004001D78681E0A2859D801A902F09CFB94
:10972000060633373B3F43474B4F5300180000F0CA
:1097300042F9062312284BD000281BD16088FFF77E
:10974000D9F90823002813D04279002A47D1264BA3
:109750001A78072312070BD5244B1A680723002A0F
:1097600006D01668002E03D0290001AAB0470300D6
:109770006A4613706B461B786088002B2AD1FFF76E
:1097800067FC06B070BD180000F06CF9D4E7180053
:1097900000F087F9D0E7180000F093F9CCE7180043
:1097A00000F0ADF9C8E7180000F0C3F9C4E71800ED
:1097B00000F0F6F9C0E7180000F0F6F9BCE7180071
:1097C00000F013FAB8E7180000F013FAB4E7072323
:1097D0006A46137069466088FFF782FFD1E7052368
:1097E000012AC5D1024BB8E78967FF1FF468FF1F44
:1097F000F868FF1FF8B52C4F8600F35904000D00E0
:10980000002B40D0DA8882423DD15A78062A33D1E3
:109810001A78002A2ED0012099681A6A097D01421F
:1098200006D0157B054203D007225A700120F8BDEF
:109830000220014204D0157B054201D00922F4E741
:109840000420014204D0127B024201D00B22ECE73B
:10985000164B1B68002BE9D05B68002BE6D020007C
:109860009847BB5900215B78122BDFD12000FFF70E
:1098700015FFDBE70E4BECE7112A04D1002900D0DD
:1098800032252900F2E7002D08D12000FFF732F938
:10989000002803D01023027913430371210028000C
:1098A000FDF798FAC2E7C046FC68FF1FF468FF1F87
:1098B000F868FF1F70B50E4E8500AB590400002BF1
:1098C00013D01B78002B11D10A4B1B68002B04D03E
:1098D0005B68002B01D02000984773595B78122BEE
:1098E00003D100212000FFF7D9FE70BD024BECE749
:1098F000FC68FF1FF868FF1FF468FF1F094B80001A
:10990000C3581020002B0CD01A6A002A09D09B687B
:10991000002B06D0127A1B7E101C9A4200D9181C0C
:10992000C0B27047FC68FF1F70B503000D00140043
:109930000220002A30D000292ED013700B78081D89
:1099400053704B789370FFF7A7FCE0700120022161
:109950002B7A23716B7B034063716A7B0A4013434C
:10996000042263716E7B1640334363716E7BF6088D
:10997000F600334363712B7B0340A371287B0140C6
:1099800000200B43A371297B0A401343A3712A7B58
:10999000D208D2001343A37170BD10B50A000100B4
:1099A0000120FFF7C1FF10BD10B50A000100022021
:1099B000FFF7BAFF10BD70B506000C000220002EA4
:1099C00030D000292ED07378201D0B70B3784B70E7
:1099D000F178FFF76DFC01223579257271794B1012
:1099E000080013409340104003438810104080004B
:1099F000C9080343C9000B436373B1794B100800D6
:109A00001340934010400343881002409200C9085D
:109A10001343C9000B4321202373FCF773FE8542D7
:109A200001D2122070BD2220257AFCF76BFE854200
:109A3000F7D823781820042BF4D86378012BF1D8B9
:109A40000020EFE7030010B50220002909D0002B09
:109A500007D00322481C0A7019000D3202F00CF9DD
:109A6000002010BD03000222080010B5002B06D014
:109A7000002904D00E32591C02F0FEF8002210001A
:109A800010BD030010B50220002909D0002B07D01B
:109A90000422481C0A7019000C3202F0EDF8002074
:109AA00010BD10B5FFF7DEFF10BD03000220002936
:109AB00006D0002B04D0052200200A701B784B70C2
:109AC000704703000220002B08D0002906D05B78E5
:109AD00000200B70013B082B00D9183070470300A1
:109AE00010B50220002909D0002B07D00622481CFF
:109AF0000A7019000A3202F0BFF8002010BD10B53C
:109B0000FFF7B0FF10BD02000B00022010B50029C6
:109B10000ED0002A0CD007211970118859701188B5
:109B2000090A997011180822D81C02F0A5F8002023
:109B300010BD03000A00022010B5002B0CD0002934
:109B40000AD099785878090201431180901CD91CD9
:109B5000082202F091F8002010BD030010B5022089
:109B6000002909D0002B07D00822481C0A701900D0
:109B7000921802F081F8002010BD02000B000220B4
:109B800010B500290BD0002A09D0092119701178CD
:109B900018185970511C062202F06EF8002010BDF2
:109BA00010B5FFF75FFF10BD02000B00022010B5DB
:109BB000002A09D0002907D05178197011180622FF
:109BC000581C02F059F8002010BD030010B5022007
:109BD000002909D0002B07D00A22481C0A7019005E
:109BE000063202F049F8002010BD10B5FFF73AFF29
:109BF00010BD02000B00022010B5002A06D000297B
:109C000004D018005178FFF753FB002010BDF0B5C9
:109C100085B017001E006A460623050008009181E2
:109C20009380FEF7C0FC1324011E02900CD0380074
:109C3000B047041E05D1280001A9FEF76FFA041EE3
:109C400002D0029802F010F82800FFF701FA200075
:109C500005B0F0BDF0B504008BB0019115000021F6
:109C6000102202A801F0F8FE334EA700B8590028D0
:109C70003CD0C388A34239D10378002B36D1427837
:109C8000062A18D102000100553235310C3006ABDE
:109C9000FFF7A9FA002829D12000FFF72FFE0200C4
:109CA00006A902A801F0E8FF200002A901F0E4FDE6
:109CB00001200BB0F0BD816E002917D00B8A112A4C
:109CC00028D19D420ED101981231093A01F0D4FEFB
:109CD000012807D1BB5920009D6EFFF70FFE290018
:109CE0000200DEE732212000FFF7D8FC2000FEF75B
:109CF00001FF061E1BD0416A002918D00B8AAB4217
:109D000015D108220198123101F0B6FE01280ED1BA
:109D1000716A0AE09D42E9D108220198123101F0EE
:109D2000ABFE0128E2D1BB59996E8A7EB9E72000CB
:109D300002F07AF8BCE7C046FC68FF1FF0B56B4D37
:109D400087007E5985B0337802900393002B00D0B2
:109D500087E0B368346A01937078062817D101222E
:109D60001B7D134202D0217B114218D102221342E3
:109D700002D0217B114251D10422134203D0237B14
:109D8000134200D08BE0019B5A7DEB5991E00738DC
:109D90000428F8D802F060F8032E42678300B36EFF
:109DA000002B03D11C2001F08FFEB066EB599C6E96
:109DB000002C1CD010220021200001F04DFE029842
:109DC000FFF79CFD01002000FFF72DFA01F034FDA4
:109DD0002082200008211230FFF725FA0298FFF7B1
:109DE0008DFDA076EB592100D888FFF70FFC0822E3
:109DF000EB591CE0B36E002B05D01A00198AF088CD
:109E00001232FFF70DFC0222019B197DEB59114222
:109E10003DD0207B10423AD0073208E0F488FCF7AE
:109E2000DBFD01002000FFF711FC0A22EB595A70FC
:109E3000029B9C002A595378073B042B11D8D088E9
:109E4000FEF758FE00284ED0C3895A08D218284978
:109E5000029B0298CB542B5941180433254801F03A
:109E6000CBFD05B0F0BDFCF79FFD03000120834250
:109E700001D100200393EB59DE88FCF79BFD039989
:109E800002003000FFF7ECFB019AEB59117D042230
:109E900011420CD0217B114209D00B22C7E7F68872
:109EA000FCF73CFD01003000FFF7EEFB6BE7019A89
:109EB000527D01210A4204D0607B084201D00C226D
:109EC000B5E702210A4204D0607B084201D00E228D
:109ED000ADE704210A4204D0627B0A4201D010227D
:109EE000A5E71222A3E7FA225200B0E7FC68FF1FA1
:109EF0000069FF1FB3A2001110B5064B1A780423A6
:109F0000100018401A4200D00348FFF727FA00203B
:109F100010BDC0468967FF1F1046FF1F70B50400C3
:109F2000FFF7D4FA051E43D12000FFF77FFA234E36
:109F3000A400A0598268937CDB0708D50321036A3B
:109F40001B790B40012B02D1017F0B430377431D8B
:109F5000D97F8B1E022B0DD8022900D00121C08889
:109F6000FCF790FF042133591A7F59700A431A777E
:109F7000280070BD01290CD102231022437000215A
:109F80000C3001F069FD305910213530FFF74BF9E5
:109F9000EEE70529ECD10223D118437010220C30D2
:109FA00001F06AFE04233259117F0B431377EAE76D
:109FB00008251828DCD1053DDAE7C046FC68FF1FFC
:109FC000F0B58BB0059143887E4F9E00F459150083
:109FD0000493002C15D1012902D000200BB0F0BD54
:109FE000101D57781678FFF757F9EB683200029387
:109FF0002B7A0499019300903B002000FCF70CFFA2
:10A00000EBE7E388049A934201D00820E6E723783F
:10A01000012B00D1D4E0059B581E092800D9CFE0C0
:10A0200001F01AFF05CE0A29CC506C859AB229009E
:10A030000498FFF773FFD1E7200029001022453074
:10A0400001F01AFEB9594B78042B02D1013B4B7039
:10A05000C3E70B000A00253335320C310498FFF7B3
:10A0600095F90498FFF702FA0522431E9841BB595F
:10A07000C0005A70B2E7200029001022553001F0CC
:10A08000FBFD049B4F4C9D00295904980A0006AB28
:10A0900055320C31FFF77AF929591022453106A8BB
:10A0A00001F0EAFC012808D10498FFF7F7F90590C0
:10A0B000002804D106222B595A7005988EE70823F0
:10A0C0000593FAE763780C2B7AD1E36E002B03D16A
:10A0D0001C2001F0F9FCE066BB59D86E00286FD057
:10A0E0001022290001F0C8FDBB590498DC6EFFF76F
:10A0F00005FC0D22A076BB595A706EE7E06E002871
:10A100005ED063780D2B5BD12B8808220382A91CBB
:10A11000123001F0B1FDBB599A68517D0222114203
:10A1200026D0186A407B104222D00C32E4E76378D4
:10A130000E2B45D1236F002B03D1162001F0C4FC58
:10A140002067BB59186F002803D01022290001F0A6
:10A1500093FD0F22BB59CFE763780F2B30D1206FCF
:10A160000622691C103001F087FDBB599A68517DA9
:10A170000422114203D0196A497B1142D5D1002132
:10A180000498FFF78BFA28E7636F002B0DD0BB59BB
:10A19000586F0028F3D01022290001F06DFD012234
:10A1A000BB5952425B6F1A61E9E7142001F08CFC45
:10A1B000BB5960675B6F002BE9D126E72978DFE7A1
:10A1C00007200BE7FC68FF1F10B5064C207001F05C
:10A1D0001BFB06212078FDF791FF0348FEF778FC72
:10A1E00010BDC0460F69FF1F6993001100200BB21C
:10A1F00070B50D00834216DA264B187801F084FB07
:10A20000041E0DD00378922B0ED0A02B37D0224BFA
:10A210001878FF283AD0210001F0E6FC002835D15B
:10A2200080200002684070BD43780E2B0BD03E2B7F
:10A23000EDD18378052B12D0082BE8D18179808865
:10A24000FFF7D8FA08E0154B82889A42DFD183687D
:10A250001878591CFEF7C0FE002817D1D7E7104B1D
:10A260001B785B0712D50F4B1B68002B0ED09B6829
:10A27000002B0BD0C289811D80889847ECE7FFF73F
:10A2800041FAA068002801D001F0EEFC200001F0A6
:10A290002BFCC5E70F69FF1F0946FF1F18200000B0
:10A2A0008967FF1FF868FF1F10B50078FFF712FAE3
:10A2B00010BD10B50078FFF7FDFA10BD0C23434325
:10A2C000084A10B59B185A68002A03D0012901D109
:10A2D000904710BD9B68002BFBD00029F9D198470F
:10A2E000F7E7C0462C69FF1F01238340094A10B5D8
:10A2F000946B1C439463506B98435063D46B200061
:10A300009843012901D120001843D063116B0B43FE
:10A31000136310BD00800040F0B500240127154BE9
:10A3200085B0DA6B144E03921A6C0192DA64019BC9
:10A33000E3403B4217D0039DE5403D400295E5B226
:10A3400002992800FFF7BAFF316A736A002908D022
:10A350003900002B01D0029979402800FFF7C4FF93
:10A3600001E0002BF9D101340C36172CDFD105B0F8
:10A37000F0BDC046008000401069FF1F064B012160
:10A380005A68C2400A4204D01B68C3401800084003
:10A3900070471B6DF9E7C046008000400122064B64
:10A3A0008240002903D0D9680A43DA607047D9682F
:10A3B0009143D960FAE7C0460038004030B5032425
:10A3C00044430F4BE25C1B199C785D7801232D1BE5
:10A3D0000135AB40013BA340A140DB430C001228F8
:10A3E00007D808499200521811681940214311609A
:10A3F00030BD054A11680B4023431360F8E7C0469F
:10A4000047C1001108F0004014F00040C21F70B5B1
:10A41000D4B20623092C0BD80125084C95400029FD
:10A4200008D00021FFF7CAFF23682B4323600023D5
:10A43000180070BD2368AB43F8E7C0460038004001
:10A44000214BF0B51B185B78022B21D10324444328
:10A450001E4A1F4EA35C12199478012215008540F4
:10A46000B76B013CE4B23D43A240B563194C1228DE
:10A4700015D89B0000290CD117495B1899680A432D
:10A480009A600123205C154A834011680B431360D6
:10A49000F0BD11495B18996891439960F1E70E4B43
:10A4A00000290DD159690A435A61225C1328E8D06A
:10A4B0000123203A93400A49086803430B60E7E709
:10A4C000596991435961F0E71069FF1F47C10011B5
:10A4D000008000408CC1001100F00040A0F000405E
:10A4E000A4F00040F8B500241B4E1C4D1C4B1B5D16
:10A4F000012B1FD1194A9269E2401A420BD0012266
:10A50000B25693402200143AD2B2022A09D8154911
:10A510004A6913434B61013402360C35172CE5D1DF
:10A52000F8BD0022B2560F499200521891680B43B1
:10A530009360F0E7022BEED1E7B23800FFF71EFF81
:10A5400001235840C1B23800FFF77AFF3800FFF707
:10A5500015FF6877DFE7C04619C100111069FF1FBA
:10A560001169FF1F00F00040012202388240054BB4
:10A57000002903D059690A435A61704759699143C8
:10A580005961FAE700380040F8B50E0001210F00CC
:10A590008740114A0400D368FD43BB43D360831E48
:10A5A0008B4201D8FFF7E0FF00212000FFF72EFFCC
:10A5B0000A4A0B4B5168012E05D139431B195160D2
:10A5C0005E700020F8BD2940516002221C196270A3
:10A5D0009A6915409D61F4E7003800400080004012
:10A5E0001069FF1F012210B58240074B002906D0D9
:10A5F00019680A431A600121FFF7C6FF10BD1968E8
:10A6000091431960F7E7C046008000400C2370B505
:10A61000002543430A4A29009B181D70094B04007A
:10A620001B185D70FFF7B0FF0123A3400649280007
:10A630000A681A430A6005490A689A430A6070BDAD
:10A640002C69FF1F1069FF1F3480004030800040DC
:10A6500070B504000E00FF2813D003250540FFF756
:10A66000D5FF084AA3089B009B183F22ED00AA4093
:10A67000AE40196820009143314319600121FFF772
:10A680008DFE70BD18380040F8B50C244443134BC0
:10A690000500E4186368002B03D1A3681220002B87
:10A6A0001AD0022201270E4B00215B195A70280094
:10A6B0002770FFF769FF63681E1E08D0A3683E007D
:10A6C000002B04D02800FFF759FE4640F6B22800C0
:10A6D0003100FFF709FE0020F8BDC0462C69FF1FBE
:10A6E0001069FF1FF7B5C420FF222B4B80001958BB
:10A6F000002491433F3A0A431A508022274F5202C6
:10A70000274E1A60274B1D5D002D21D0A31E012B63
:10A7100003D80121E0B2FFF727FF012D18D11F4B0D
:10A720009B69E3402B4213D0E3B218000193FFF77B
:10A7300025FE01000198FFF755FFE3B2143B022B01
:10A740001DD801217156184A8D405369AB4353619E
:10A750003B7F002B0DD0E5B22800FFF795FF2800C6
:10A76000FFF70CFE7B7F0100834202D02800FFF739
:10A77000A5FD01340C370236172CC3D1F7BD0121DA
:10A7800000237156F3568D40074A9B009B189A6828
:10A79000AA439A60DCE7C04600E100E01069FF1FB1
:10A7A00019C100111169FF1F00F0004010B501210F
:10A7B0000400FFF7E9FE0123044A002011194B7041
:10A7C000A34091690B43936110BDC0461069FF1F00
:10A7D00070B50E0015000400FFF718FF0C2363434B
:10A7E000094A20009B189D605E60FFF74DFFF02135
:10A7F000064B074A8900051E5A5002D02000FFF779
:10A8000005FF280070BDC0462C69FF1F0000FF1F18
:10A8100019A3001170B5134D07202C78002C1FD1FF
:10A82000982221005200280001F00EFB0123C420D1
:10A83000FF222B700C4B80001C635C630B4B1C6075
:10A840005C600B4B195891433F3A0A431A508022DF
:10A8500052021A600D20074A074901F07DFA2000D4
:10A8600070BDC0461069FF1F00800040A0F000408E
:10A8700000E100E0E5A60011E5A40011030010B519
:10A880000620072B09D8054A137001F0E5F9D721F6
:10A890000020034B034A89005A5010BD3846FF1F61
:10A8A0000000FF1F151BFF1F70B51D0002240C299F
:10A8B00010D8094ACA40D2070CD5FBF72FFF041E57
:10A8C00008D1059A04992800FBF744FFFCF7B2FD74
:10A8D000FFF712FB200070BD1210000030B50D789C
:10A8E00002232C009C43184201D02B431C00082556
:10A8F0002300AB43284201D02B00234320241D001A
:10A90000A543204201D01C4325002A230D70184284
:10A9100004D011781E3B0B43137030BD0028FCD1CE
:10A920000C2113788B43F7E7F8B51D0006AB1B88A5
:10A93000140007AA0E000B201778002B27D10A78E5
:10A94000022A49D14A68507811780002244A084303
:10A950008018042840D801F07FFA03121D1B230041
:10A96000F06801F0A9F8021CC0B2B84200D93A1C44
:10A97000D2B22000F1682A8001F07EF906E00222BE
:10A98000F3681B882A8023701B0A63700020F8BDBF
:10A990000622EEE701232B80F3681B782370F5E78E
:10A9A000F368002B16D008222A801A8822701A8891
:10A9B000120A62705A88A2705A88120AE2709A8843
:10A9C00022719A88120A6271DA88A271DB881B0AE6
:10A9D000E371DBE72B80D9E701202B80D7E7C04666
:10A9E00000D6FFFFF7B516000A781D0008AB1F88D8
:10A9F0000C000123022A18D14A685078117800020D
:10AA00002B4A0843801803280FD801F025FA0225A5
:10AA10004439E06801F050F8C0B20723B84204D3CB
:10AA20007B190193152B02DD0D231800FEBDE06894
:10AA30002A003100C01901F01FF96B4600209B88E5
:10AA4000E268D0541B4B1B68834203D01B688342CF
:10AA500000D098470023E8E70B23002FE5D1022D13
:10AA6000E2D1737832781B021343E2681380114BF2
:10AA70001B68002BEED01B68002BEBD00120E8E711
:10AA80000B23002FD1D1062DCED12A003100E06852
:10AA900001F0F2F8DEE70B23002FC6D1012DC3D160
:10AAA00032787533012AC0D8E3681A70D2E7C046FD
:10AAB00000D6FFFF1C6BFF1F70B50C0015000728A8
:10AAC00037D801F0C9F9041436361B36242E182065
:10AAD00015290BD8184E16220021300000F0BCFFBB
:10AAE00022002900300001F0C7F8002070BD1820B6
:10AAF0000229FBD11288114B1A80F6E71820082989
:10AB0000F4D10A000E48290001F016F8EDE71820EC
:10AB10000129EBD10B4B10780B49DA69FFF7DEFE08
:10AB2000E3E718200129E1D1064B10780749DA6BD9
:10AB3000F4E70220DAE7C046046BFF1FB646FF1FAA
:10AB4000AC46FF1F3C46FF1F6446FF1F8446FF1FA5
:10AB5000030010B50020DB0704D50721024A034893
:10AB600000F08CF810BDC046A4C100113C46FF1F88
:10AB7000054A03001068002803D082889A4201D158
:10AB8000806870470068F6E7206DFF1F0A880300A1
:10AB900008009A4204D08A8804309A4200D00020EB
:10ABA00070470000F8B5F82200230D4F0D4E79686C
:10ABB000050042433370994200D07B600A4C00216B
:10ABC000200000F049FF00231A007C60AB4202D154
:10ABD00000203370F8BD01332280DBB2F834F5E792
:10ABE000206EFF1F1C6EFF1F246DFF1F73B56B4689
:10ABF00001900600684615001980FCF74DFF041E01
:10AC000011D1002D0FD07689002E11D00C2000F02C
:10AC10005BFF00280ED0084A0460136886808560B8
:10AC2000002B02D11060200076BD1A001B68F7E7E8
:10AC30000224F8E71324F6E7206DFF1F012100220C
:10AC40000A4B10B549420A4C198099809A719A7042
:10AC5000084B2070012019805A60FFF7A3FF20786D
:10AC6000FCF778FF0448FDF733FF10BD246BFF1F8E
:10AC7000286EFF1F206EFF1F29AD0011022310B5A3
:10AC8000002802D0FFF7B2FF0300180010BD00003B
:10AC9000030010B50020DB0704D50421024A034855
:10ACA000FFF7A4FF10BDC046B8C10011BC46FF1F8E
:10ACB000F0B50E2687B003930CAB1F8802ABF618D5
:10ACC0000500080031000292FDF768F80400012039
:10ACD000002C0FD03088FFF74BFF03000E20002B15
:10ACE00008D05E68002E05D021002800039B029A40
:10ACF0000097B04707B0F0BD0A4B10B5984207D196
:10AD00000122002352420A808B708A808B7110BD11
:10AD1000FFF73CFF0028FAD001235B4203800023A9
:10AD20008370F4E7FFFF0000F8B5050001290AD1A0
:10AD3000134E00243388F827AB4219D0280011495C
:10AD4000FFF7DAFF06E0022904D10139FDF73EFFE3
:10AD50000028EDD0F8BD3B0063437268D018D35A89
:10AD6000002B09D03A00002100F076FE0134E4B255
:10AD7000054B1B78A342EED801235B423380DDE70D
:10AD8000206EFF1F246BFF1F1C6EFF1F10B5FFF707
:10AD9000FDFE03000020834200D0987810BD000023
:10ADA000F0B589B01C000EAB80CB03901E8810ABB1
:10ADB0001B78049202930B7A0D00DB0616D42B78D5
:10ADC0000593022B24D00498FFF7D2FE002812D05E
:10ADD00003689C46002B0ED0029B220001932900A1
:10ADE0003B00644603980096A04705E00498FFF7EF
:10ADF000BFFE002802D10E2009B0F0BD8368002BF1
:10AE0000F9D00A222900039898470028D7D0F3E701
:10AE10006B6858781A786B4B000210439842D2D86E
:10AE2000043B984210D2684B984242D015D8674BE9
:10AE3000C0180128C7D80B20002EDDD1EB681A7886
:10AE400059683A80200028E0614BC018032800D9D7
:10AE500079E001F001F8846A789E5E4B9842B2D1A5
:10AE60000B20002EC8D101233B80EB6831001B78FA
:10AE700023706889013080B2FCF790FF3A88031E86
:10AE80000ED0017802328A183A8042896270428973
:10AE9000120AA27059680278E01C00F0EDFE06E08C
:10AEA00004323A8031000422601C00F0D5FD0020FD
:10AEB000A2E70B20002E9FD1EB6807A91E88042370
:10AEC0003B80330A300026706370FCF767FF051E75
:10AED00028D004AB9A890E2304A95B183E49C668A2
:10AEE000FCF7D0FF00280BD12B783C486A68059905
:10AEF000FBF786FB002803D1012304AA5B42D38120
:10AF00003278022A06D17168201D00F0B5FE3B8818
:10AF100002333B800E2304AA9B181B88A3701B0AD4
:10AF2000E370C4E704ABDE81F4E70B20002E00D011
:10AF300062E7E9680398FFF729FF02233B8020704E
:10AF4000000A6070B3E70B20002E00D054E7022205
:10AF5000EB681B883A8023701B0A6370A7E7E868D8
:10AF600000F0AAFDC2B203000720B24200D243E7BC
:10AF70000DD00299DBB27118994202DB921BD3B259
:10AF80000293029BE9681A003B8089195AE7002363
:10AF9000F6E70B20002E00D02EE70722EB683A8060
:10AFA0001A7822705A7862705A88A2705A88120AE7
:10AFB000E2701A792271DA886271DB881B0AA37148
:10AFC00075E7C046042900000228000000D8FFFFF2
:10AFD000FFD6FFFF03280000FFFF0000E8C00011BC
:10AFE000F0B58DB06B460020089120229B5E834215
:10AFF0003DDAA64B187800F087FC071E32D00378A4
:10B00000B02B2CD10079023816281FD800F004FD8F
:10B0100017001E001E001E0031001E0096001E00BC
:10B020001D011E0052011E0073011E00CD011E00F5
:10B0300050021E001E001E008E021E00E302944BF2
:10B0400094491B8878880B80FBF71AF83800FCF7C6
:10B050009BFF914B1B68002B01D0380098473800AC
:10B0600000F042FD8020089B0002434018000DB014
:10B07000F0BDF6220021874800F0EEFC0BAA3B7BD6
:10B080007989388900923A000D32FCF79FFD04005F
:10B09000804B1B78002C3FD146E0804B788805938D
:10B0A0007F4B4100CB5A0BAE073BDBB23288029399
:10B0B000002301937B4B210006930093059BFFF730
:10B0C0006FFE744D002810D1069B3A8A1B889A4265
:10B0D0000BD138000599123000F0CEFC002804D0C6
:10B0E0002B7862899B00EB185A80162306A81B1840
:10B0F000328820007989FCF7C5FE2B7804009A007D
:10B10000AA1851880029C3D00133DBB22B70002864
:10B1100007D006A9C98A9180634A12889A42BCD88E
:10B1200002E0012149429180002B04D059497888DE
:10B13000FAF7DAFF8AE73E890A2479E000253E899A
:10B14000574B06937B88069A5B009B5A033B9D42B4
:10B1500002DB002DF0D05BE0162206A812183B7B24
:10B16000798900923A0030000D32FCF72FFD0590EE
:10B17000002858D04689017A7888FCF7F1FC041E33
:10B1800044D1464B78880793069B4100C95A454BEA
:10B190000439C9B206AAD28A069302910194009397
:10B1A0000599079BFFF7FCFD041E2FD1069B39492B
:10B1B0001A88931C002D26D14B807988384B490082
:10B1C000CB5A5119033B8B4220DD059B31485B89EB
:10B1D00041190B71A91C0135C9B2EDB20591451990
:10B1E0001B0A2B71059B2D490433181800F044FDF0
:10B1F0002C4B059A1B88D318DDB22C4B9E4205D0F0
:10B200000136B6B29CE749889942D6D0002D0CD0C1
:10B21000204C2800618800F06FFC207021007888A5
:10B22000FAF772FF12E7059CF0E7002C00D183E7E4
:10B230007B78142B00D109E716493B794E800B70BF
:10B240000C717888FAF712FF00E7162406ABE418B1
:10B2500021003889FCF7A2FD011E00D1B7E17888F2
:10B2600022880F4C45002C5B0A4D013CE4B202944D
:10B2700000240F4B01940095FFF792FD041E00D0AF
:10B2800014E129007888FAF74FFFDFE6286EFF1FE8
:10B29000A845FF1F2C6BFF1F206BFF1F266CFF1F95
:10B2A0005C67FF1F1C6DFF1FA645FF1FFFFF00000F
:10B2B0002E6BFF1F162406ABE41821003889FCF71B
:10B2C0006DFD011E00D182E178882288AE4C4500D8
:10B2D0002C5BAE4D013CE4B202947C89AC4B0194F2
:10B2E0000095FFF75DFD041E00D0DFE0290078889F
:10B2F000FAF724FFAAE60025A44B1D803B00FE338D
:10B300001B78A24A78880792AB4208D99E4B1288D4
:10B310000693069943005B5A013B9A4203DB079967
:10B32000FAF716FF92E616246B00FB18059306AB9E
:10B33000E418059B21001889FCF730FD011E03D19C
:10B34000059B01241E8973E77888924B2288069C0E
:10B35000099343001B5B904E013BDBB20293002339
:10B3600000960193099BFFF71BFD041E02D0059B6D
:10B370001E895DE77B88069A5B009B5A079A1088B6
:10B3800032881218934202DC1B1A013B33807F4C37
:10B39000023032880999001900F06EFC2388328847
:10B3A00001359B182380EDB2A8E70BAA3B7B798976
:10B3B000388900923A000D32FCF708FC0025059010
:10B3C000059B002B04D10A24002D00D16EE060E023
:10B3D000059B7888197AFCF7C3FB0100041E63D132
:10B3E000694C6C4B788806940993069B4400E45A98
:10B3F000694B063CE4B20BAE32880793029401918C
:10B4000000930599099BFFF7CBFC041E4CD1079BC9
:10B410005E491B881A1D002D30D14A80059B5B4C6C
:10B420005A8963191A716B1C9BB2E318120A1A71BC
:10B43000162306A832881B1879890598FCF722FD87
:10B44000FF21AA1C2E1D03350B00059092B2B6B247
:10B45000ADB2002803D006ABDB8AD9B21B0AA21812
:10B46000651911712B714C4D301D2A8849492018DE
:10B4700000F002FC2B88F618B5B2A1E7498891428A
:10B4800007D17A8806995200525AEB18053A9A4227
:10B49000C4DC3E4C2800618800F07EFA2070210058
:10B4A0007888FAF75FFED1E5002DF2D13E89BFE63C
:10B4B000162606ABF61831003889FCF76FFC3D0004
:10B4C0000400FF3500282DD0037A9B060CD40022FF
:10B4D0007B893989788800923A000C32FFF7E8FBC3
:10B4E000041E10D03E8915E03088FFF741FB00288C
:10B4F0001AD08368002B17D0210012227888984731
:10B50000041EE4D0EEE7AB78002B02D17888FAF77E
:10B5100039FE0026AB78002B00D097E5002C00D137
:10B5200094E585E60124DDE70E24DBE7162506AB6E
:10B53000ED1829003889FCF731FC041E47D0037A46
:10B540009B0611D4154A7B881188994203D0144870
:10B55000814207D11380134BF8261D780023D9B2FE
:10B56000A94221D30924A1E72888FFF701FB00287D
:10B570002FD08368002B2CD0210012227888984786
:10B58000041EDFD092E7C0465C67FF1F2C6BFF1FD5
:10B590002E6BFF1F266CFF1F1C6DFF1F206EFF1FF1
:10B5A000FFFF00001C6EFF1F310059435468013338
:10B5B0006018615A0029D2D13C0008342100F822D9
:10B5C00000F05AFB21007888FAF7E4FD3EE50124FB
:10B5D0006CE70E246AE71D4B1A887B889A4231D0AB
:10B5E0007888FAF7E1FD31E5F8230598516843437F
:10B5F000CD18C95A00291FD03B7A012B0BD16C887A
:10B60000AB887888AA1D0094FFF752FB041E02D075
:10B6100000233B722E88F8220021280000F01CFA3B
:10B6200000232B80059B0133DBB20593084B059962
:10B630001B78064A8B42D7D801235B421380002C2B
:10B64000CED0F5E5002634000596EFE7206EFF1F0B
:10B650001C6EFF1F70B504000E001500FFF796FA70
:10B66000031E08D131000548FFF790FA03001120AE
:10B67000002B02D01C8000209D7070BDFFFF0000D9
:10B68000F8B50B4F06003B780D001400FF2B0ED0D1
:10B690000A2000F0F9F8011E09D0B123038000232D
:10B6A00046800371C5800481387800F09DFAF8BDAA
:10B6B000FD46FF1FF7B50F0008A90600088809A975
:10B6C0000B240988002821D10234022B1ED1557881
:10B6D00013782D021D432B008B4301937334002BF1
:10B6E00014D1FB68300019000093FFF74FFB019C59
:10B6F00085420BD02A0030000099FFF7ABFF041EF3
:10B7000004D12A0030007989FFF7BAFF2000FEBD7E
:10B71000F0B50E7885B003900AA805880120022EA6
:10B720000DD14C682778647824023C43054FBC4215
:10B7300005D10398DBB201960095FFF7BBFF05B07A
:10B74000F0BDC0460229000010B504000C4800F00E
:10B750005BFA0C48A16B00F057FA0B48E16B00F064
:10B7600053FA0A48216C00F04FFA094B094819684E
:10B7700000F04AFA084B1B68002B00D09847FEE700
:10B780009ABF0011B0BF0011BFBF0011CEBF0011A2
:10B7900004ED00E0DDBF00112C6EFF1F002307B594
:10B7A00001A80193FFF7D0FF044A0548002110B516
:10B7B000121A00F051F9F8F703F9FEE7306EFF1F97
:10B7C0000047FF1F0000000001B40248844601BC8E
:10B7D000604700BF4532FF1F01B40248844601BCE8
:10B7E000604700BF156B010001B40248844601BCEC
:10B7F000604700BF5118FF1F01B40248844601BCD6
:10B80000604700BF8552010001B40248844601BC74
:10B81000604700BFC926000001B40248844601BC4D
:10B82000604700BFA13BFF1F01B40248844601BC32
:10B83000604700BFC9A9000001B40248844601BCAA
:10B84000604700BF2951010001B40248844601BC91
:10B85000604700BF6571010001B40248844601BC25
:10B86000604700BF8B52010001B40248844601BC0E
:10B87000604700BF014C010001B40248844601BC8E
:10B88000604700BF311B000001B40248844601BC80
:10B89000604700BF1D4D010001B40248844601BC51
:10B8A000604700BF055E000001B40248844601BC49
:10B8B000604700BF5D17000001B40248844601BC28
:10B8C000604700BF75A9000001B40248844601BC6E
:10B8D000604700BFC95C010001B40248844601BC56
:10B8E000604700BFB53CFF1F01B40248844601BC5D
:10B8F000604700BFB54C010001B40248844601BC5A
:10B90000604700BF8D12000001B40248844601BCAC
:10B91000604700BFF54E010001B40248844601BCF7
:10B92000604700BF2D38FF1F01B40248844601BCA8
:10B93000604700BFC94A010001B40248844601BC07
:10B94000604700BFE139FF1F01B40248844601BCD3
:10B95000604700BFB352010001B40248844601BCF5
:10B96000604700BFF94C010001B40248844601BCA5
:10B97000604700BF2124000001B40248844601BC96
:10B98000604700BFC56D010001B40248844601BC98
:10B99000604700BF691F000001B40248844601BC33
:10B9A000604700BF090E000001B40248844601BC94
:10B9B000604700BFE117000001B40248844601BCA3
:10B9C000604700BF851F000001B40248844601BCE7
:10B9D000604700BF3555000001B40248844601BCF1
:10B9E000604700BFF30E000001B40248844601BC6A
:10B9F000604700BF350E000001B40248844601BC18
:10BA0000604700BFA946010001B40248844601BC5A
:10BA1000604700BF5D38FF1F01B40248844601BC87
:10BA2000604700BFD93DFF1F01B40248844601BCF6
:10BA3000604700BF9DA9000001B40248844601BCD4
:10BA4000604700BFB930FF1F01B40248844601BC03
:10BA5000604700BF5147010001B40248844601BC61
:10BA6000604700BF154D010001B40248844601BC87
:10BA7000604700BF456B010001B40248844601BC29
:10BA8000604700BFCD4C010001B40248844601BCB0
:10BA9000604700BF5549010001B40248844601BC1B
:10BAA000604700BF4550000001B40248844601BC15
:10BAB000604700BF5125000001B40248844601BC24
:10BAC000604700BFDD52010001B40248844601BC5A
:10BAD000604700BF3D4B010001B40248844601BCF1
:10BAE000604700BF1D4B010001B40248844601BC01
:10BAF000604700BF434D010001B40248844601BCC9
:10BB0000604700BF350E000001B40248844601BC06
:10BB1000604700BFED4A010001B40248844601BC01
:10BB2000604700BF3938FF1F01B40248844601BC9A
:10BB3000604700BFD53AFF1F01B40248844601BCEC
:10BB4000604700BF810E000001B40248844601BC7A
:10BB5000604700BFADAE000001B40248844601BC9E
:10BB6000604700BF893CFF1F01B40248844601BC06
:10BB7000604700BF9D32FF1F01B40248844601BCEC
:10BB8000604700BF2D39FF1F01B40248844601BC45
:10BB9000604700BF613BFF1F01B40248844601BCFF
:10BBA000604700BF7918000001B40248844601BC18
:10BBB000604700BF2526000001B40248844601BC4E
:10BBC000604700BF291C000001B40248844601BC44
:10BBD000604700BF5952010001B40248844601BCCD
:10BBE000604700BF213BFF1F01B40248844601BCEF
:10BBF000604700BF594F010001B40248844601BCB0
:10BC0000604700BFC521000001B40248844601BC62
:10BC1000604700BFE53A010001B40248844601BC18
:10BC2000604700BF4551010001B40248844601BC91
:10BC3000604700BFE928000001B40248844601BC07
:10BC4000604700BFF535FF1F01B40248844601BCC0
:10BC5000604700BF0124000001B40248844601BCD3
:10BC6000604700BF151BFF1F01B40248844601BC9A
:10BC7000604700BFD949010001B40248844601BCB5
:10BC8000604700BFE94C010001B40248844601BC92
:10BC9000604700BFE93AFF1F01B40248844601BC77
:10BCA000604700BFE548000001B40248844601BC7B
:10BCB000604700BF0189000001B40248844601BC0E
:10BCC000604700BFC534FF1F01B40248844601BC71
:10BCD000604700BF1147010001B40248844601BC1F
:10BCE000604700BF7D18FF1F01B40248844601BCB5
:10BCF000604700BF8534FF1F01B40248844601BC81
:10BD0000604700BFD91B000001B40248844601BC53
:10BD1000604700BFEDA5000001B40248844601BCA5
:10BD2000604700BF5522000001B40248844601BCB0
:10BD3000604700BF3D18000001B40248844601BCC2
:10BD4000604700BF5D32FF1F01B40248844601BC5A
:10BD5000604700BF017F000001B40248844601BC77
:10BD6000604700BFE532FF1F01B40248844601BCB2
:10BD7000604700BFA54F010001B40248844601BCE2
:10BD8000604700BFB13DFF1F01B40248844601BCBB
:10BD9000604700BFC53F000001B40248844601BCB3
:10BDA000604700BF0D3CFF1F01B40248844601BC40
:10BDB000604700BF090E000001B40248844601BC80
:10BDC000604700BF056A000001B40248844601BC18
:10BDD000604700BF6D30FF1F01B40248844601BCBC
:10BDE000604700BF4D1F000001B40248844601BCFB
:10BDF000604700BFB14E000001B40248844601BC58
:10BE0000604700BFC51D000001B40248844601BC64
:10BE1000604700BF6DBC000001B40248844601BC0D
:10BE2000604700BF0D52010001B40248844601BCC6
:10BE3000604700BF091B000001B40248844601BCF2
:10BE4000604700BFDD66010001B40248844601BCC2
:10BE5000604700BFB70E000001B40248844601BC31
:08BE6000604700BFC53DFF1F54
:10BE6800000201030202030304030502060207029B
:10BE7800080209030A030B030C020D000E030F034B
:10BE8800100311031303140315001600B53D001128
:10BE9800E93D00110000000002000000AABE0011E8
:10BEA800192A0F1809000000F1590000FD240000AC
:10BEB800D9810011EDA1001141760011DD7F00113B
:10BEC800C1540011E1AF001129510011A53F001123
:10BED800D540001100000000161600000200000006
:10BEE800F0BE0011F4FFF3FFD2FC00001542001170
:10BEF8000000000000000000547579610042312EF6
:10BF0800330030303134006769746875622E636FAE
:10BF18006D2F7076767800544830350002000000A6
:10BF280038BF0011292A282A272A262A252A242A1E
:10BF38000A180000E20400007102000078EC00001A
:10BF4800744000001027000060F000000664000044
:10BF5800204E000000000000050000001F501D00DA
:10BF6800023CB4000001150013000000A10200000B
:10BF78003031323334353637383941424344454617
:10BF8800005048592B36325858504C55533035309C
:10BF980034005B48617264206661756C7420686166
:10BFA8006E646C65725D0A004C522020203D203082
:10BFB80078253038780A0050432020203D203078FA
:10BFC800253038780A0050535220203D20307825FB
:10BFD8003038780A0049435352203D2030782530C4
:10BFE80038780A00C55800111959001100000000DE
:10BFF8000200000004C000116F2A6E2A1A18EAD83D
:10C00800BC80F0FC60000000000000000000F303AA
:10C01800B59747D6F613F7D777E6F0A7F47400007C
:10C0280001A00000000000006410B71DC8206E3B8E
:10C03800AC30D9269041DC76F4516B6B5861B24D27
:10C048003C7105502083B8ED44930FF0E8A3D6D691
:10C058008CB361CBB0C2649BD4D2D38678E20AA0F9
:10C068001CF2BDBDFB349B5F800000800010000007
:10C078000000000043620011CD78001167620011D2
:10C08800D57C0011EB620011AB7C001161630011DB
:10C09800817C0011B3630011497E00111B640011FB
:10C0A800497E00114D640011037E00116163001187
:10C0B800397C0011D9630011E17D001100000000F6
:10C0C80000000000BF640011E17D0011216500112E
:10C0D800E5780011052A042A012A002A02290328E2
:10C0E80001280028011800180000000000000000C6
:10C0F80000000000000000870101020102010102A6
:10C108000102030304010301010101010303020108
:10C1180003000D000E0010001100130014010701A8
:10C1280008010A010B011C011D0204020502070295
:10C13800080219021A021C021D0301030203170058
:10C148000201000504000807000B0A001716001D6D
:10C158001C010201010504010E0D01111001141347
:10C16800011716011A19020201020B0A020E0D022A
:10C178001110021413021716030504030807030B12
:10C188000A030E0D0001020307090A0B0E0F101116
:10C1980012141718191A1B1F2021220029A900118F
:10C1A800E5A900110000000002000000EEC0001127
:10C1B8000000000011B7001100000000020000009C
:04C1C800ECC00011B6
:020000041FFFDC
:1000000000000000113F0011B0BE0011ACBE001195
:100010000C64FF1F00000000000000000000000052
:1000200000000000000000000000000000000000D0
:1000300000000000000000000000000000000000C0
:1000400000000000000000000000000000000000B0
:1000500000000000000000000000000000000000A0
:100060000000000000000000000000000000000090
:100070000000000000000000000000000000000080
:100080000000000000000000000000000000000070
:100090000000000000000000000000000000000060
:1000A0000000000000000000000000000000000050
:1000B0000000000000000000000000000000000040
:1000C0000000000000000000000000000000000030
:1000D0000000000000000000000000000000000020
:1000E0000000000000000000000000000000000010
:1000F0000000000000000000000000000000000000
:1001000000000000000000000000000000000000EF
:1001100000000000000000000000000000000000DF
:1001200000000000000000000000000000000000CF
:1001300000000000000000000000000000000000BF
:1001400000000000000000000000000000000000AF
:10015000000000000000000000000000000000009F
:10016000000000000000000000000000000000008F
:10017000000000000000000000000000000000007F
:10018000000000000000000000000000000000006F
:10019000E934FF1F3133FF1FC1660100000000007A
:1001A000000000000000000000000000000000004F
:1001B000000000000000000000000000000000003F
:1001C000000000000000000000000000000000002F
:1001D000000000000000000000000000000000001F
:1001E000000000000000000000000000000000000F
:1001F00000000000000000000000000000000000FF
:1002000000000000000000000000000000000000EE
:1002100000000000000000000000000000000000DE
:1002200000000000000000000000000000000000CE
:1002300000000000000000000000000000000000BE
:1002400000000000000000000000000000000000AE
:10025000000000000000000000000000000000009E
:10026000000000000000000000000000000000008E
:10027000000000000000000000000000000000007E
:10028000000000000000000000000000000000006E
:10029000000000000000000000000000000000005E
:1002A000000000000000000000000000000000004E
:1002B000000000000000000000000000000000003E
:1002C000000000000000000000000000000000002E
:1002D000000000000000000000000000000000001E
:1002E000000000000000000000000000000000000E
:1002F00000000000000000000000000000000000FE
:1003000000000000000000000000000000000000ED
:1003100000000000000000000000000000000000DD
:1003200000000000000000000000000000000000CD
:1003300000000000000000000000000000000000BD
:1003400000000000000000000000000000000000AD
:10035000000000000000000000000000000000009D
:10036000000000000000000000000000000000008D
:100370009DB7001100000000000000000000000018
:10038000000000000000000000000000000000006D
:10039000000000000000000000000000000000005D
:1003A000000000000000000000000000951AFF1F80
:1003B000000000000000000000000000000000003D
:1003C000000000000000000000000000000000002D
:1003D000000000000000000000000000000000001D
:1003E000000000000000000000000000000000000D
:1003F00000000000000000000000000000000000FD
:081838003072FF1F4118FF1F71
:10184000024981F3088802F023FC00003072FF1F78
:1018500010B502F0A5FC072804D0122808D00228F1
:1018600008D010BD044A0420136B01331363F8E75A
:101870000220F6E71420F4E70468FF1FF8B507001C
:101880000C0026002500503630785135002804D150
:101890000300287058342370F8BD2978CA00481E08
:1018A0008141A3183800A25C5B68C9B2FFF7D0FF82
:1018B00000280DD12B78DA00A218013350602B706C
:1018C0003378044A013B3370136A01331362D8E75B
:1018D0000123DFE70468FF1F5C234343074910B57A
:1018E000C9180B0058331B78012B05D1FFF7C6FF31
:1018F000034A936A0133936210BDC0463868FF1FE4
:101900000468FF1F10B502F0E3FA064A0121130034
:1019100010CB4942D967044B136002F049FC200008
:1019200010BDC04600E100E01000100010B504003A
:1019300002F0CEFA024B1C6002F03AFC10BDC04629
:1019400000E100E010B5040002F0C2FA4021094AAB
:10195000200013688B43136002F0C2FC01F0A6FD67
:101960000022054B01201A60044B04321A6002F079
:1019700057FAFEE71CF00040C4F00040C0F0004001
:10198000431E5A425341A022F0B5D2015B4213409C
:10199000154D164A40019B182A18127E8BB00191F2
:1019A000002A1BD01A000832D46F0022E6B206AF1C
:1019B000E4B294420EDC2818C369002B08D00199C8
:1019C00002AA117106AA049202AA167303A89847E4
:1019D0000BB0F0BD1978B9540132EAE71A7D1A78D4
:1019E00006AB01261A70E6E7C46AFF1F00400040FC
:1019F000F0B5254B04004001C25C85B0002A2BD015
:101A00001A18117E002927D0917E002924D011793F
:101A1000022921D11689D788D168F51BADB22A1CBD
:101A2000102D00D9102292B2BE4217D118180123EE
:101A300003710023C269C38003819A4206D06846BD
:101A4000032103730171029301A890470820002C21
:101A500000D0192001F022FC05B0F0BD013C654228
:101A60006C41A0256442ED012C40084D1B186419FF
:101A7000074D0633013A92B2AA42EDD01888461CAF
:101A80001E80085C2070F5E7C46AFF1F004000401C
:101A9000FFFF00000F220E4B10B59868104002386F
:101AA0000A280BD802F08EF90D0A0B0A0A110A0A4D
:101AB0000A0A060002210020FFF762FF10BD012183
:101AC000F9E70020FFF794FFF8E7DB6FF6E7C04681
:101AD000004000400F220E4B10B5986810400238AD
:101AE0000A280BD802F06EF90E0A0B0A0A120A0A2B
:101AF0000A0A060002210120FFF742FF10BD012162
:101B00000800F9E70120FFF773FFF7E7DB6FF5E760
:101B10000090004013B5334C2378072B3DD8324B4F
:101B20001A78324B002A39D18022196852020A43AE
:101B30001A60252001F0F4FF20232D4A11680B4381
:101B4000802113606B460422C905086807331042E0
:101B500028D080210422C905C86810422ED08021D7
:101B60002020C905CA688243CA6014221A701A78F4
:101B7000002A2FD18021C905C86820320243CA60DB
:101B800014221A701A78002A28D11A4B1A7D22784A
:101B90005A601D221A705932DA6013BD1A6816494C
:101BA0000A40C5E7086802430A6014221A701A78CE
:101BB000002ACED01A78013AD2B2F7E7C8680243B9
:101BC000CA6014221A7019784A1ED2B21A700029FB
:101BD000F9D1C4E71A78013AD2B2C7E71A78013AC4
:101BE000D2B2CEE73846FF1F0047FF1F3CF000404F
:101BF0003046FF1F00200040FFFFFEFF564B70B530
:101C00001B68012B03D1554A936D0133936502F094
:101C1000FFFA534B534A1860534B544C1A6001233C
:101C2000534A1360534A13602378002B06D00622D0
:101C30005149524802F004F900232370504A514B95
:101C400010681B78C1B2002B0ED14F4CC0B2237864
:101C50005BB2002B4FDB237824785BB264B21B04A9
:101C600024021B191B1813600B1C50294ED950233A
:101C7000464A47491078DBB2FF2202284BD1086858
:101C8000444C454D267890432A78964254D9227880
:101C900024782E78023B5D10A31B6B435201D31AAC
:101CA00010335B111843086002F0C2F8031F012BC8
:101CB00045D83A4B1B78002B06D0394B1B78002BAC
:101CC00002D0002002F0D4FAA122364B920099787B
:101CD000354B4A431B689B18832292009B181B7844
:101CE000033B012B03D8AF20400002F019F9012279
:101CF0002E4BDA8270BD237824785BB264B2FF3356
:101D0000FF341B0424021B190138ABE7CAB2022AB4
:101D1000AED20223ACE70868254C264D26789043C6
:101D20002A78964208D9227824782D78023B5B10D5
:101D3000641B63435201B2E72378DBB2B2E70228A7
:101D4000D5D11D4B1B78013B022B03D91B4B1B78B4
:101D5000022BCCD16C20C8E79809FF1FFC0FFF1F96
:101D60003C67FF1FFF3F0000141003404067FF1F48
:101D70000C10034000100340D50BFF1F7211FF1F12
:101D8000B40003408C09FF1F680AFF1F490AFF1FA8
:101D900094000340460AFF1F470AFF1FF908FF1F70
:101DA0002209FF1F300DFF1F3409FF1FBC0BFF1F4F
:101DB000440AFF1F450AFF1F1C09FF1F2309FF1FBD
:101DC00010B502F06DF90022014B1A8010BDC0461B
:101DD0003867FF1F10B502F083F9A121054A890079
:101DE0009478054A61431268044B5218528C1A8049
:101DF00010BDC046300DFF1F3409FF1F3867FF1F9D
:101E000010B50D4B0D4A9978A1239B004B431268E6
:101E1000D218531DD97F0A4B1B88994209D2441C02
:101E200007D0C82805D0D2695B1A5A43054B5343E3
:101E3000C01802F01DF910BD300DFF1F3409FF1F3F
:101E40003867FF1F7102000070B5244D2B68002B0E
:101E500028D002F0BDF82B68D8402B680400002B76
:101E600027D002F01DFA2B68D8401D4B1D4A9978E7
:101E7000A1239B004B431268D118D25C91239B0095
:101E8000002A20D0CA580132CA50174B17491B6884
:101E90000868834214D3D23B181A012A1AD0144B73
:101EA000186070BD02F094F8124B196802F008F93E
:101EB000D3E702F0F5F90F4B196802F001F9D4E706
:101EC0000D495B18E8E7CA500C4B1B68DB68E41847
:101ED000201AE4E7F530FF30E1E7C0461C08FF1F99
:101EE000300DFF1F3409FF1F9C09FF1F3C67FF1FB8
:101EF000A009FF1F1808FF1F2DFF3F004467FF1FA9
:101F000070B504000D00282916D10300A433C2883F
:101F10001B889B1A0B4A9BB293420DD906006A3666
:101F200005223100653002F093F9002804D1310018
:101F3000200002F0ADF970BD2900200002F080F809
:101F4000F9E7C046FE7F0000F8B50400012002F06A
:101F500077F902F02DF8174A17491060174D030062
:101F6000886A174E28607568AC46164D2F680025A4
:101F7000BC4501D275687D1B134E00193560C862DF
:101F8000A4204C6A40032043486210490978002984
:101F900005D00F490978022902D10F3B1360F8BD23
:101FA000012901D1083BF9E7032901D1053BF5E7F8
:101FB000033BF3E7E408FF1F00F00040340AFF1F73
:101FC00028100040180AFF1F1C0AFF1F1C09FF1FD2
:101FD0004A0AFF1F70B580241025E405A3682B432F
:101FE000A36002F0ADF8A368AB43A36070BD00002E
:101FF000F7B5160080221C001023D20501919168CC
:1020000005000B43936000225A4BD7301A6002F050
:102010005FF89D232A002F009B00EB58CA32012154
:102020000092FC37002B01D00021009A386801F0A3
:102030001FFF2900009BCB311A784F4BD3351A6014
:102040004B780A781B0213438A7812041A43CB7820
:102050001B061343494A1BBA13604B790A791B02CA
:1020600013438A7912041A43CB7931001B061343B8
:10207000434A1BBA13606B782A781B021343AA7871
:1020800012041A43EB781B0613433E4A1BBA136033
:10209000019A330213433C4A13603C4B22001B1B42
:1020A0009C4603293DDCB3089A0013005142B21A42
:1020B000032A46D1354AE018511A82784078120432
:1020C00000020243E05C043302430A600022FF2B5B
:1020D0004BDDF0222E4B12011A600F222D4B1A609D
:1020E0002D4A1368002BFCD00023224A2749136095
:1020F000091B321D0B191B68043A180A2370607003
:10210000180C1B0EA070E3700434002AF2DC80224D
:1021100010213B68D20501333B6093688B43936089
:10212000F7BD6346D578981893782D061B042B438A
:10213000157804392B43557804322D022B43036064
:10214000AFE7022A0AD1114AE05C511AE21852782C
:10215000120202430A6004339BB2B7E7012AB5D1E9
:102160000A4A521AE15C1160F5E7084959180A60F9
:102170000433ACE7000004403C0004403800044055
:1021800034000440300004400C00044000010440CE
:10219000040004401000044014000440F7B515008A
:1021A00080221C001023D2050091916807000B4388
:1021B00093600023654AD730136001F089FF9D23A7
:1021C0003E009B00F9583B00CA363200FC33002920
:1021D00000D07FE0586801F04BFE390032785C4B4C
:1021E000CB311A604B780A781B0213438A78AC46CD
:1021F00012041A43CB78281D1B061343554A1BBAF9
:1022000013604B790A791B0213438A7912041A432B
:10221000CB791B061343504A1BBA13604B7A0A7AD8
:102220001B0213438A7A12041A43CB7A21001B063D
:1022300013434A4A1BBA1360009A2B021343484ABD
:1022400013602200474B1B1B0093009BCE785B184A
:1022500001938B7836061B0433430E7804383343DE
:102260004E78043136023343019E33600328ECDCA0
:102270000321A808431C9B002940800003292BD17F
:102280003849E5185E18A9786D78E35C09042D02D9
:10229000294319433160030008330021FF2B2DDD52
:1022A000314B324919600F21314B19600123274905
:1022B0000B60304B19680029FCD006211B680B40CD
:1022C000042B20D080220020D20593680A318B4352
:1022D0009360FEBD01217DE7022908D121495D18E7
:1022E000E1184978E35C090219432960D3E7012921
:1022F000D3D11C495918E35C0B60CCE71948181876
:1023000001600433CAE7002310490B606346002BC9
:102310000CDC3B00FC335A68102101325A608022E9
:10232000D205936801208B439360D2E7009B9B18F2
:102330001B68190A13705170190C1B0ED3700423FB
:102340005B4291709C440432E0E7C04600000440C8
:102350003C00044038000440340004403000044095
:102360000C0004400001044004000440080F000079
:10237000100004401400044070B5061E19D002225B
:10238000614B9B799343012B13D1604B1A78FF2A41
:102390000FD15A78FF2A0CD19A78FF2A09D1DA781E
:1023A000FF2A06D11A79FF2A03D15B79FF2B00D1CE
:1023B000A7E0574B0C201A78012A08D00022554D6F
:1023C0001A702B781A00093A042A01D8212070BD0E
:1023D0005A1F012AFAD94C4CA07B042800D990E05E
:1023E000A279032A00D98CE0821E012A03D86288D0
:1023F0001F2A00D885E0002E61D0012E00D080E099
:10240000A288012AE2D0002B0AD10138032803D880
:1024100001F0D8FC151D19151F202E7001F070FE5B
:102420002B785A1E032A16D800253B4B1D60282303
:10243000237501F065FFA8422ED0A580C6E70223D0
:1024400020202B70EAE7042322202B70E6E70323E9
:1024500021202B70E2E7073B012BB7D82F4B1B68DD
:10246000DB6A9B06B2D52E4B1A78002AAED1A27B2E
:10247000911E012901D9002AA8D1022280211A70B7
:102480002823284D89012878237501F011FE802129
:102490002878890101F014FF0123A380224B1B78C7
:1024A000002B0AD0FA228021204B92001B880902BF
:1024B0005A431C4B187801F02BFD002087E701F0F0
:1024C00007FD2B78A680073B012B06D918482E70F4
:1024D00001F0A6FE1E2001F013FE114B114C1A78DC
:1024E000002A06D080210022207889011A7001F08C
:1024F000DFFD01F05DFE80212078090201F0D8FDAA
:10250000DBE7122063E7C046A60BFF1F6B09FF1F26
:102510001A09FF1F1C09FF1F4809FF1F4467FF1FFF
:102520002309FF1F1B09FF1F2109FF1F2C09FF1F84
:102530000010004010B5002901D001F0A9FC10BD29
:10254000F7B5604B01919978A1239B004B435E4AFC
:10255000060014681022E418D6235B00E0583623E6
:10256000FF33E35C00279343222B41D1574B0F3AB3
:102570001A600760012501F03BFE019B1880E823EB
:102580005B00E35C002B01D0B34258DD0023504FC9
:10259000FB70AD33FF33E3581A68002A03D09B88E1
:1025A000DB439B071DD03823FF33E35C002B18D09F
:1025B0009B235B00E35C002B13D1D133FF33E35C3F
:1025C000B3420EDAA4235B00E15AE018090A023193
:1025D00001F08EFC23000122FE33013E01351A87F3
:1025E000FA70E8235B00E35C002B2AD0A8B2FEBDA2
:1025F00003683D00002BBED081880430090A0231F7
:1026000001F076FCD6235B00E3581F60B2E723009D
:10261000B133BA00FF339858013781880430090A72
:10262000023101F065FCE8235B00E35CBB42EEDCB9
:10263000E822F61AED1800235200A354A6E700275B
:10264000F1E7200001F034FE00281FD0002E1DDD30
:102650007319882647190193B600200001F090FCF9
:102660005A30800020184068013581880430090AFA
:10267000023101F03DFC200001F07AFDA359013345
:10268000A351BD4202D0019B9D42E6D1114BE35CB8
:10269000002BABD095239B00E35C002BA6D00E4B08
:1026A000E15A0029A2D00D4AA35C994202D9013314
:1026B000A3549BE700231A212000A35401F098FBA8
:1026C00094E7C046300DFF1F3409FF1F001403407C
:1026D000E010FF1F5A020000720200005E020000BC
:1026E000F8B51D4B1D4F1A78002A10D1BA7B002A6D
:1026F00002D101321A7003E0032AFAD0022AF8D07C
:1027000001F0FEFD00220120154B1A70F8BD154B9B
:10271000154D1C68154B9E7801232B702878C0B28C
:1027200000F0CEFCBB7B002B0BD101F099FDA12367
:102730009B007343E41883239B00E41823782B70D9
:10274000E4E7032B02D101F0B3FBF0E70020022BFA
:10275000DCD101F055FDEAE71C09FF1FA60BFF1FA6
:102760002309FF1F3409FF1F490AFF1F300DFF1FF8
:10277000F0B587B00EAD2F780FAD2D780593AC4630
:10278000634614000E4D0CAA12782E7803930D9B0D
:10279000009201932200059B029701F0F1FC2E703C
:1027A000012C01D0042C08D1802206498B88934348
:1027B000054A1278D20113438B8007B0F0BDC046A2
:1027C0001C09FF1F6C11FF1F7809FF1F0B001B3B2B
:1027D00070B504003020E02B0DD81300E025493BF4
:1027E000FF3B9BB2ED00AB4205D8034B20001982A2
:1027F0005A8201F0A5FB70BD8410FF1F10B501F0D7
:1028000007FD054B00205B68052B04D9034A52687D
:10281000D20200D4980810BD00100040FCE100E096
:1028200070B501F055FB0D4B1B68FC33DC691D6A6C
:10283000FFF7E4FF6419844204D2094B01241B68AA
:10284000002B07D004220024064B1A70064A936915
:102850000133936101F0ACFC200070BD4467FF1FA1
:102860009809FF1F2309FF1FFC0FFF1F70B50C4DB8
:102870002B68FC335C6A01F02BFBFFF7BFFF2B6872
:102880000025FC339B6AE318834204D2054B1B6886
:10289000AB4200D1051B01F08BFC280070BDC04687
:1028A0004467FF1F9809FF1FD722044B92009B58D3
:1028B00010B5002B00D0984710BDC0460000FF1F88
:1028C000F0B587B001F008FAFFF7EEFFC54BC64C34
:1028D00004931B78022B45D1C44B1B68186A01F086
:1028E000AFFCC34BC34A1A60C34BC44A1A60A02250
:1028F000C34B52001A60049B187801F001FBC149D8
:10290000C14801F06DFCC149C14801F069FC1022C9
:10291000C04BFF201A60802252031A60802292036B
:102920001A60802212041A6001F0A2FC012001F05A
:10293000F7FBFA20400001F0A3FB582001F0F0FA69
:10294000B54801F06DFB012001F062FB072001F0AA
:10295000DFFCE26DB14B1A4084235B001343E36557
:1029600007B0F0BD01F0F4FBAD4E0290322001F053
:1029700067FC33681B0628D43C2001F061FC0F2063
:1029800001F05EFC974B1B78012B00D113E18025F1
:1029900033682B4200D0A1E0636C03202B436364B7
:1029A00001F04EFC01F0D4FB029B0299C31A5A1E9F
:1029B000814200D81A009B4B1A608C4B19681E2369
:1029C0005343994A9B18CB618BE701F0C1FB8023ED
:1029D000E26BDB0213430390E363E26D8F4B032052
:1029E0001A4028231343E36501F02AFC0320A56E57
:1029F00001F026FCA36E0320DB03DB0B019301F047
:102A00001FFCA76EED03FF03ED0BFF0B874AAB180E
:102A1000C22B2ED8019B9B18C22B2AD8BB18C22BC5
:102A200027D8019B2A009D4200D21A00019B9D429B
:102A300000D91D003B00974200D21300BD4200D9CF
:102A40003D005B1B122B14D80C22336814209343D7
:102A500033603368764A1340336001F0F1FB08219C
:102A6000A36EE26DDB038A43E265724ADB0B1360FF
:102A700085E7032001F0E4FBA36EDB03DB0B05938A
:102A800001F066FB039B0399C21A531E814200D8D2
:102A90001300694A93421BD9FF23356864492D0A04
:102AA0001D4032686B1C1B060A401B0C134333602D
:102AB0000C23326800209A43083B1343336001F033
:102AC00067FB5E485E4BA840984205DCFEF73AFF84
:102AD000019D0197059F99E75A48F7E700235A4E51
:102AE00033608023226CDB0213432364636C032076
:102AF0002B43636401F0A4FB33680133336080230C
:102B0000626C5B021343636405230193E26D434BE4
:102B100003201A404D4B1343E36501F091FB08215C
:102B2000A26EE36D434F8B43E3653B6802394B4331
:102B3000D203D20B9A420CD89B1A3B2B0BD8E36DD5
:102B400043490B40E365636C0B406364414B1A607F
:102B500028E7D31AF1E7019B013BDBB20193002B7D
:102B6000D4D1E36D3A4A1340E365636C1340636468
:102B70003368042B07D9BFF34F8F374B374ADA60DE
:102B8000BFF34F8FFEE7636C0320AB43636401F038
:102B900057FBE26D214B03201A4028231343E365C2
:102BA00001F04EFB0822A36EDB03DB0B3B60E36D01
:102BB0009343E3659AE70722E36B1340012B02D1AD
:102BC000002001F09DF9264D264AAB6802201340F3
:102BD000AB6001F035FB8023AA685B001343AB6058
:102BE000E0E6C0464A0AFF1F00F000404467FF1FAE
:102BF000000003400180063DBC0003403408000093
:102C0000A40003407102000014100040FFFF3F00C9
:102C10002810004000E100E03075000000FEFEFFDB
:102C2000C4F000402C67FF1F7206000091FCFFFFFC
:102C3000FF00FFFF3467FF1FE30C0000E880000087
:102C40005F361E0060361E009C45FF1F28000100F5
:102C5000FFFFFEFF3067FF1F00ED00E00400FA05F4
:102C60003CF00040FFFEFFFF694E336888331B686D
:102C700083F3088801F03CFA00F018FC654B664AC3
:102C80001B68934207D0002001F082FA0221634AB8
:102C900013688B431360FFF713FE614B614C187888
:102CA000C0B201F0FDF80023A3600233A3605E4BC5
:102CB0000120236001F0C4FA0323A36001F048FA65
:102CC000040001F0A5FA050001F042FA574B186024
:102CD00001F096F9564B1968621A531EA14200D2B0
:102CE00013008022D203934201D39B029B0A3268D5
:102CF000D16AC90700D478E04E491C0C09689BB220
:102D00004C4359432402090A641803274A49FC32F8
:102D100093680A6849489B1A494A4A4E12684A49C8
:102D20009B18414A34609A183B400193036892080B
:102D30009C46019B0A6063440360042B03D9013263
:102D40003B400A6003600B684049E418200001F032
:102D5000B7F93F4F3D493B68C3183B6020000193E2
:102D600001F0DEFA3B4C20680818384920608842A0
:102D700005D9019B01333B6001F0D2FA216001F0DB
:102D80006FF8354B1B78002B0ED001F041FA3168FB
:102D9000324B4A1B1B6812189A4233D2591A4919EE
:102DA000091A2F4801F01CFA2E4C237A002B0FD061
:102DB00001F02EFA3168E3684A1B1218934224D9B5
:102DC000591A4919091A284801F00AFA00232372EE
:102DD000264B83F3088801F0C3F8022001F090F934
:102DE000002001F0D5F901F023F9DC01990002344B
:102DF000641A5900641A09214B438033CB40A4085C
:102E0000E41882E7FA218900CBE71949DBE7C046DD
:102E10004467FF1F0C0AFF1FB6412103100000404A
:102E2000490AFF1F14100040C4090000100AFF1FC8
:102E3000340AFF1F380AFF1F200AFF1F280AFF1F3E
:102E40001C0AFF1F2867FF1F240AFF1F71020000D2
:102E50006008FF1F2C0AFF1F1C09FF1FE408FF1F4B
:102E600000100040740BFF1F3C10004000000020C9
:102E7000DC050000A022054B92009B5810B5002BEA
:102E800001D0984710BD01F053F9FBE70000FF1F88
:102E9000A122054B92009B5810B5002B01D09847FA
:102EA00010BD01F045F9FBE70000FF1FA222054B12
:102EB00092009B5810B5002B01D0984710BD01F02F
:102EC00037F9FBE70000FF1FA322054B92009B5838
:102ED00010B5002B01D0984710BD01F029F9FBE790
:102EE0000000FF1FA422054B92009B5810B5002B39
:102EF00001D0984710BD01F01BF9FBE70000FF1F50
:102F000070B501F085F9514B1860042001F0F8F814
:102F100000F0B6FF0400C30702D401F029F870BD29
:102F200000224B4B1A604B4B1878013804282CD8E0
:102F300000F048FF03231B1F2700200001F0A0F929
:102F40000128ECD0444C2378042B71D100F0F0FF21
:102F5000002806D000F0C4FF582000F0E1FF022353
:102F60002370032001F0CCF8D9E7200001F0B0F97C
:102F7000E6E7200001F024F9E2E7200001F010F874
:102F8000DEE7200001F064F8DAE700F051FF050009
:102F9000012808D1314B1B78053B012B03D82000B9
:102FA000FFF768FFCEE72C4B1B78022B01D0052BD7
:102FB00020D1022D28D12A4B9B7BAB431CD1200072
:102FC000FFF766FF254B18780128BBD16405B9D4FB
:102FD000234925224B7B034205D1233A13405A4211
:102FE000534126331A000B7D9342ABD9322001F0B6
:102FF0001FF9A7E7022D07D1184B1B78052B11D11C
:103000002000FFF753FFDDE7012D0BD1012B03D18A
:103010002000FFF759FF95E7062B03D12000FFF7AB
:1030200061FF8FE7200001F083F8022D8AD1C9E704
:10303000032B04D10B4B987C00F0DAFF91E7072BB0
:103040008FD1094B987B00F03BFF8AE79C09FF1F5B
:103050009809FF1F9009FF1F2309FF1F1C09FF1F6D
:10306000A60BFF1FBC0BFF1FD40BFF1FFA210A4B3F
:103070000A4A49001A640A4A5A500A4A04395A50FC
:10308000094A08319A64094A5A50094A5C315A502F
:10309000084ADA667047C0460000FF1F7127FF1F0D
:1030A0006D28FF1F2128FF1F7923FF1FE126FF1F27
:1030B000011EFF1FD51DFF1F10B500F06BFE10BDD8
:1030C0008023F7B59C46264B264F01932649274A75
:1030D000274D284C284B02281AD1604638600868D2
:1030E000264E304080263603304308600199097827
:1030F000002909D11660224A2A60224A2260E02271
:1031000019689143A03A1BE08021C9021160F2E7DF
:1031100066463E600F68194E3E408027FF023E43E0
:103120000E600199097800290DD1176001280ED190
:10313000154A2A60154A2260E02219689143C03A74
:103140000A431A60F7BD802189021160EEE7E02191
:103150000F4A02432A600F4A22601A688A43F0E746
:103160004B0AFF1FE0000340D800034090000340DB
:10317000000003405000034040000340FFFFE3FF16
:103180000280063D804508220180063D80660822B7
:103190000080069880550822F8B51E4B80261A68D4
:1031A000002014003440324232D11A681A4F3243A0
:1031B0001A6001223B68063093433B6001F040F8FF
:1031C0000122164D2B681E432E603B680A261343CE
:1031D0003B608027BF00124B1B683B4211D1013E70
:1031E000F6B2FF2E09D17E220E4B1C682B68E40B31
:1031F0001440934323432B6005E0082001F020F89E
:10320000E9E7002EEFD180222B68600893432B6002
:10321000F8BDC046C4F000405CF0004018F000402B
:1032200068F0004060F0004010B500F099FF012107
:103230005820034A00F0D4FEFFF7AEFF10BDC04691
:10324000600AFF1F10B578220021034800F0A0FE9D
:1032500000F006FF002010BD4C6AFF1F70B504008F
:1032600000F036FE00230C200B4A010059438D1854
:10327000515C00290DD0A14208D1012300246B70BC
:1032800000F0C6FD00F094FF200070BD01330A2B52
:10329000EBD11224F6E7C0464C6AFF1F70B504005C
:1032A00000F016FE002319001D000D4A10780028BA
:1032B00006D0A0420CD1557001310C320A29F5D14B
:1032C000002B0AD100F0CCFE00F072FF002070BD90
:1032D0005078461EB0411B18EEE700F099FDF3E769
:1032E0004C6AFF1FF7B504000C20002384460E4DE6
:1032F000019267465F43E85D7E19A04212D0002824
:103300000BD10A4B9C4662461B7808331370019B15
:1033100070707C557160B360FEBD01330A2BE8D13B
:103320000320F9E70720F7E74C6AFF1F486AFF1FF1
:103330008020F8B5484BC0051B68C1248360474B0B
:10334000FF251A68012313434361454BA4001A6803
:10335000444B40211A60444B1A68444B1A60444B5A
:103360001A59AA431A51C52292009E58AE433143BE
:10337000802699509F583F49F6010F403E439E508A
:103380009E5880273602360A3043985080201A59BA
:1033900000020A4002431A5104341A59364E3F04BF
:1033A000324080263A431A511A5936061202120A3E
:1033B00032431A5108341A5980260A4002431A51DE
:1033C000C32292009F58B446AF4337439F509F5843
:1033D000294E0F4007439F509F58374080263604A0
:1033E000374380269F509F5836063F023F0A374397
:1033F0009F50C0221F59AF433A431A511A59120223
:10340000120A1643C6221E5192009C58AC436546D0
:103410002C439C509C5800250C4020439850C720BA
:1034200080001A58154C1140C02212020A431A504B
:10343000134B1B78DB08AB4201DC0020F8BD23787E
:10344000002B06D0A368002B00D0984701350C3420
:10345000EEE71220F2E7C0463446FF1F3046FF1F5A
:10346000B0F00040446AFF1FB4F00040406AFF1F04
:1034700000E100E0FF00FFFFFFFF00FF4C6AFF1FBD
:10348000486AFF1F030010B51F2809D80722002033
:103490001340072404490A78A24313430B7010BD5C
:1034A00000230620F5E7C046486AFF1F034A044987
:1034B000136800200B4013607047C0461CF00040AA
:1034C000FFFFC1FF054B06491B780A6805485B07EB
:1034D00002401B0B134300200B607047486AFF1F1C
:1034E0001CF00040FFFFC1FF70B50C25FFF7EAFF9D
:1034F0000A4B1C780A4BE4086543ED18002C01D1F7
:10350000200070BD2B78002B06D06B68002B00D0FC
:103510009847013C0C3DF1E71220F2E7486AFF1F93
:10352000406AFF1F1FB5002102220B00019100918C
:10353000052000F00DFD02230B490A681A42FCD158
:1035400020230393039B5A1E0392002BFAD1074AB0
:103550001368002BFCDA0B246C442000012100F0DE
:1035600077FC207804B010BD90C8004000C800402F
:1035700013B504000A4B0193019B002B01D11120CC
:1035800016BDFFF7CFFF23000340044205D00520FE
:1035900000F056FE019B013BEDE71800F0E7C04646
:1035A000FFFFFF0707B500F093FC80220821D2053A
:1035B000936A0191002B01D10739916202210C4AD3
:1035C00011600199481E01900029FAD10331116060
:1035D000053101910199481E01900029FAD111602D
:1035E000002B02D18022D205936200F0E1FD07BDDD
:1035F00000C00040F0B52D4C89B02378002B4FD18E
:10360000FEF780F902232A4F03903A681A42FCD150
:1036100020230693069B5A1E0692002BFAD1254EB4
:103620003368002BFCDA0120FFF7A2FF011E02D055
:10363000112009B0F0BD030003220190009005ADF8
:103640009F2000F085FC0321280000F001FC0223EC
:103650003A681A42FCD120230793079B5A1E07920F
:10366000002BFAD13368002BFCDA0120FFF780FF32
:103670000028DDD10398FEF759F9AA786B78110478
:103680001B020B4329780B4363601300113B0A496B
:10369000052B07D801239340A3600B6001232370FF
:1036A0000020C6E780231B03F6E7C0461C46FF1F29
:1036B00090C8004000C800409808FF1F1E4B30B55E
:1036C0005A6818781D4B85B0D31859424B410121D7
:1036D0000093002300F07CFD194B1A4A02259A63DF
:1036E00000221A6510325A658022C4219D65164B4E
:1036F0001648D202DA6789004258154B80241A40D6
:1037000080231B0413434350642341200393E405A7
:1037100000F006FA402000F003FA6562039D6B1E7C
:103720000393002DFAD103236362FFF73BFFA562E9
:10373000FFF760FF05B030BD2846FF1F95FFFEF77D
:1037400000C80040050001FF04E100E000E100E0E6
:10375000FFFF00FFF0B585B00700FEF7D3F80223A6
:1037600005002D4C22681A42FCD120230093009BB7
:103770005A1E0092002BFAD1284E3368002BFCDA37
:103780000120FFF7F5FE002803D01124200005B02A
:10379000F0BD234B2360022322681A42FCD1202370
:1037A0000193019B5A1E0192002BFAD13368002B22
:1037B000FCDA0120FFF7DCFE0028E6D1194B1F6080
:1037C000022322681A42FCD120230293029B5A1E34
:1037D0000292002BFAD13368002BFCDA0120FFF7AC
:1037E000C7FE0028D1D1104B2360022322681A4261
:1037F000FCD120230393039B5A1E0392002BFAD182
:103800003368002BFCDA0120FFF7B2FE041EBCD1A6
:103810002800FEF78BF8B9E790C8004000C80040C8
:1038200001000006A8C800400180000110B500207A
:10383000FFF790FF10BD000010B5064B18705960DF
:10384000FFF73CFF00211320034AFFF74BFD002048
:1038500010BDC0462846FF1FBD36FF1FF0B504004F
:1038600085B003920291FEF74DF8882263035B0B4B
:1038700052051A438023DB059D6A8023274F00925F
:10388000BA68002601901B039A420CD9F82326003F
:103890001B041E401C4206D08022214B52025E6255
:1038A00019680A431A60002D0BD100F011FB0222A7
:1038B0001C4B1A608023DB055A62013A9A6200F0C1
:1038C00077FC0023039A934220D1002D0AD100F007
:1038D000FFFA144B03221D608023DB055A629D62B0
:1038E00000F066FC8023BA681B039A4208D9002EB8
:1038F00006D000220A4B0C495A621A680A401A6024
:103900000198FEF713F8002005B0F0BD009A029967
:10391000D2181278CA540133D4E7C0461C46FF1FA0
:1039200000C8004000C00040FFFFFEFFF0B587B0B8
:10393000029103920400FDF7E5FF019000F0C8FA40
:10394000802302250122234EDB0535605D629A62E9
:1039500000F02EFC204F3B682B42FCD12023049327
:10396000049B5A1E0492002BFAD11C4D2B68002B8D
:10397000FCDA0120FFF7FCFD002802D0112007B07F
:10398000F0BD2000039A029900F03AFA02230400E5
:103990003A681A42FCD120230593059B5A1E0592D2
:1039A000002BFAD12B68002BFCDA0120FFF7E0FD99
:1039B000051EE3D100F08CFA80230322DB0535607D
:1039C0005A629D6200F0F4FB0198FDF7AFFFE0B290
:1039D000D5E7C04600C0004090C8004000C8004085
:1039E000F0B5802489B00600FDF78CFFE405A36ADA
:1039F00002250393029000F06BFA0123304F3D60E3
:103A00006562A36200F0D4FB2E4C23682B42FCD1EC
:103A100020230593059B5A1E0592002BFAD12A4DAF
:103A20002B68002BFCDA0120FFF7A2FD002803D051
:103A30001124200009B0F0BD244B2360022322682A
:103A40001A42FCD120230693069B5A1E0692002B95
:103A5000FAD12B68002BFCDA0120FFF789FD021E4A
:103A6000E6D11B4B03211E60030001900090202033
:103A700000F06EFA022322681A42FCD12023079339
:103A8000079B5A1E0792002BFAD12B68002BFCDAF9
:103A90000320FFF76DFD041ECAD100F019FA802340
:103AA0000322DB053C605A629C6200F081FB039BB1
:103AB000002B01D1FFF776FD0298FDF737FFB8E73D
:103AC00000C0004090C8004000C80040010000064F
:103AD00094C8004007B5000201910422000A01A920
:103AE000FFF724FF0EBD000073B5050005240B4A47
:103AF000A3005B429B1819686B46DE1D300000F086
:103B000007FB022804D133782B55013CEFD276BD58
:103B1000052CFCD00128FAD10230F8E71409001175
:103B20001F2807D8012380228340D20591680B43C8
:103B3000936070473F2808D80123802220388340B3
:103B4000D20551690B435361F3E75F28F1D8012394
:103B5000802240388340D205116A0B431362E8E7A4
:103B60001F2807D8012280218240C9058B68934312
:103B70008B6070473F2808D801228021203882407E
:103B8000C9054B6993434B61F3E75F28F1D80122E4
:103B9000802140388240C9050B6A93430B62E8E7F5
:103BA0001F2810D880230200DB05153A1968012A66
:103BB00006D820229143196019680A431A60704799
:103BC00001228240F6E73F2811D880230200DB055E
:103BD000353AD968032A06D810229143D960D968AA
:103BE0000A43DA60EBE7012220388240F5E75F28DC
:103BF000E5D842238022181A413B8340D205516AFE
:103C000099435162516A0B435362D8E710B50400DF
:103C1000012813D1A022184992050B685B015B09AA
:103C200013430B60154B164A19681140154A0A4395
:103C30001A60402219680A431A6010BD0028FCD19E
:103C400001000A2000F0BCF921000B2000F0B8F9B7
:103C5000C0220A4B920019680A4340211A601A6870
:103C60008A431A60B022044912060B685B015B09A3
:103C700013430B60E1E7C04614F000401CF0004025
:103C80007F00FEFF80FD010072B6074A1368013312
:103C900013600422054B1A600023054A136080223A
:103CA000D2055360FEE7C0467808FF1FC0F0004011
:103CB000C4F00040044B054A1A60054B1A6000220C
:103CC000044B1A607047C046140AFF1F841E000090
:103CD000380AFF1FC4F000400023034A1360034A60
:103CE0001360034A1360704754F0004040F10040F5
:103CF00044F10040002310B5184C8AB000930193A2
:103D00002378012B27D06946012000F0F1FA002822
:103D100017D1009B12490293019B06AA0393114BF2
:103D200002A81B680493104B1B68059300F008FA67
:103D300010220E4906A800F08BFA002804D1FF23B8
:103D4000237000200AB010BD0123094A074902A8C8
:103D5000237000F0F5F90120F4E7C0464867FF1F23
:103D600010290011082900110C2900112029001127
:103D70004C67FF1F13B501246946012000F0B8FA13
:103D8000034B00940193FFF7B5FF200016BDC0461A
:103D9000BB0B000010B5FFF79FFFFFF7EBFF0028FC
:103DA00002D0024B984710BDFEE7C046E1A20000DA
:103DB00002B4714649084900095649008E4402BCC4
:103DC0007047C04602B4714649084900095C490081
:103DD0008E4402BC7047C04603B471464908400097
:103DE0004900095A49008E4403BC70470000000096
:103DF00001B40248844601BC604700BF53B90000CB
:103E000001B40248844601BC604700BF95730100BD
:103E100001B40248844601BC604700BF21A90000EC
:103E200001B40248844601BC604700BFA1AF000056
:103E300001B40248844601BC604700BFDD0C0100AC
:103E400001B40248844601BC604700BFE94C010050
:103E500001B40248844601BC604700BF3D710100C7
:103E600001B40248844601BC604700BFD54401004C
:103E700001B40248844601BC604700BF21440000F1
:103E800001B40248844601BC604700BFBD0B01007D
:103E900001B40248844601BC604700BFE9D4000079
:103EA00001B40248844601BC604700BF8914010088
:103EB00001B40248844601BC604700BF75F80000A9
:103EC00001B40248844601BC604700BFC1F700004E
:103ED00001B40248844601BC604700BF75A90000D8
:103EE00001B40248844601BC604700BF6DF6000083
:103EF00001B40248844601BC604700BFC1150100FF
:103F000001B40248844601BC604700BFEDA5000033
:103F100001B40248844601BC604700BF8B520100D7
:103F200001B40248844601BC604700BF7912010019
:103F300001B40248844601BC604700BF01D70000BD
:103F400001B40248844601BC604700BF116E000006
:103F500001B40248844601BC604700BF496D0100BE
:103F600001B40248844601BC604700BF7997000055
:103F700001B40248844601BC604700BFDD0A01006D
:103F800001B40248844601BC604700BFD9B00000BC
:103F900001B40248844601BC604700BFB70E000070
:103FA00001B40248844601BC604700BFF5350100FA
:103FB00001B40248844601BC604700BFBD5C0100FB
:103FC00001B40248844601BC604700BFBDA3001194
:103FD00001B40248844601BC604700BFE90B010000
:103FE00001B40248844601BC604700BF016701007C
:103FF00001B40248844601BC604700BF4DF900008F
:1040000001B40248844601BC604700BFC16601009C
:1040100001B40248844601BC604700BFE5120100BC
:1040200001B40248844601BC604700BF8D11010005
:1040300001B40248844601BC604700BF85520100BC
:1040400001B40248844601BC604700BF51B800007B
:1040500001B40248844601BC604700BFF935010045
:1040600001B40248844601BC604700BFADAE000009
:1040700001B40248844601BC604700BF8937010093
:1040800001B40248844601BC604700BF85120100AC
:1040900001B40248844601BC604700BFA9B70011C3
:1040A00001B40248844601BC604700BF8D82000015
:1040B00001B40248844601BC604700BFB35201000E
:1040C00001B40248844601BC604700BF090E0000ED
:1040D00001B40248844601BC604700BF8944000027
:1040E00001B40248844601BC604700BFF9ED0000FE
:1040F00001B40248844601BC604700BFC9A9000062
:1041000001B40248844601BC604700BF19070100A2
:1041100001B40248844601BC604700BF99380011D1
:1041200001B40248844601BC604700BF6911010028
:1041300001B40248844601BC604700BFE917010092
:1041400001B40248844601BC604700BFDD3F000067
:1041500001B40248844601BC604700BF156B0100F2
:1041600001B40248844601BC604700BFED6801000D
:1041700001B40248844601BC604700BF5976010083
:1041800001B40248844601BC604700BF9D6A00003C
:1041900001B40248844601BC604700BF016C0100C5
:1041A00001B40248844601BC604700BFE927000013
:1041B00001B40248844601BC604700BF9DA90000CD
:1041C00001B40248844601BC604700BF05340100C9
:1041D00001B40248844601BC604700BFC56D0100C0
:1041E00001B40248844601BC604700BF2D6C010049
:1041F00001B40248844601BC604700BFCD0C0100F9
:1042000001B40248844601BC604700BF19FA0000AF
:1042100001B40248844601BC604700BFC95C01008C
:1042200001B40248844601BC604700BFC1A500003C
:1042300001B40248844601BC604700BF61370100F9
:1042400001B40248844601BC604700BF01890000F8
:1042500001B40248844601BC604700BFCD4C010058
:1042600001B40248844601BC604700BFE9F6000083
:1042700001B40248844601BC604700BFED6B0100F9
:1042800001B40248844601BC604700BF013401000C
:1042900001B40248844601BC604700BF85C10000EC
:1042A00001B40248844601BC604700BF6D0B0100A9
:1042B00001B40248844601BC604700BF71B00000F1
:1042C00001B40248844601BC604700BF0D520100A2
:1042D00001B40248844601BC604700BF09340100B4
:1042E00001B40248844601BC604700BFF9A6000043
:1042F00001B40248844601BC604700BFE1AC000045
:1043000001B40248844601BC604700BFA9D8000040
:1043100001B40248844601BC604700BFF90D0100AA
:1043200001B40248844601BC604700BF090E00008A
:1043300002000000EAC0001101000000A0BE001150
:1043400002000000E6C00011010000007043FF1FE2
:1043500002000000A8BE0011010000008C64FF1FD5
:1043600002000000E4C00011030000000064FF1F11
:104370001200000002000000EAC00011010000006D
:10438000E4BE001102000000E6C0001101000000C0
:10439000E1BE001102000000EEBE001103000000AB
:1043A0003B64FF1F02000000E4C000110300000096
:1043B0005064FF1F02000000E6C000110100000071
:1043C000E0BE001102000000ECBE0011030000007E
:1043D0001164FF1F02000000E4C000110300000090
:1043E0003264FF1F02000000EAC00011010000005B
:1043F00024BF001102000000E6C00011010000000F
:10440000B944FF1F0200000036BF00110100000088
:104410001FBF001102000000E6C0001101000000F3
:10442000B844FF1F0200000034BF0011010000006B
:104430005864FF1F02000000E6C0001101000000E8
:10444000B744FF1F0200000032BF0011010000004E
:104450000FBF001102000000E6C0001101000000C3
:10446000B644FF1F0200000030BF00110100000031
:104470000ABF001102000000E6C0001101000000A8
:10448000B544FF1F020000002EBF00110100000014
:1044900005BF001102000000E6C00011010000008D
:1044A000B444FF1F020000002CBF001101000000F7
:1044B00000BF001102020202020200000000000020
:1044C00016150000514D0011174D001178BF001155
:1044D00090011D0018001800FFFF070102030405EA
:1044E00006020106000000000000000000000000BD
:1044F00000000000000000000000000000000000BC
:104500000300000002000000EAC0001101000000EA
:10451000F8BF001102000000E6C000110100000019
:104520007445FF1F0200000002C0001101000000DE
:104530008664FF1F02000000E4C0001103000000B9
:10454000F066FF1F02000000E6C00011010000003D
:104550007445FF1F0200000000C0001101000000B0
:104560008864FF1F02000000E4C000110300000087
:10457000E866FF1F12A6A6A60000000000000000CB
:10458000161500000001000000000111FFFF0000EF
:1045900050485936000000000000000001000000F3
:1045A00089BF00110B000500F7000000B4000028CF
:1045B000002800283075A000A000A000A00000087E
:1045C0000008E001F00010001000100010001000C2
:1045D000100050005000500010001000D0070000E4
:1045E000000000000F0001000500307507001000FA
:1045F000010081FF00000000FF000000A575001110
:10460000AD7300113D710011FFFF0100FF000000BC
:10461000C19F00113D9D0011559C0011000000003C
:104620000000000000000800040000003B0001083A
:104630005902E00188212800FF000000020000006C
:10464000EAC0001101000000B0C10011020000002A
:10465000E6C0001101000000B946FF1F0200000083
:10466000E2C0001101000000046BFF1F0200000007
:10467000E6C0001101000000B846FF1F0200000064
:10468000E0C0001101000000B646FF1F020000005C
:10469000E6C0001101000000B446FF1F0200000048
:1046A000DEC0001101000000AC46FF1F180018001A
:1046B0001D00900102000003020200000200000041
:1046C000EAC0001101000000C4C100110200000096
:1046D000E6C0001101000000FC46FF1F02000000C0
:1046E000DCC000110000000000000000020000001B
:0E46F000E4C0001103000000246BFF1F20FF38
:040000051FFF184180
:00000001FF
